:100000000C94BB010C94CD010C94CD010C94F02EFA
:100010000C94E02B0C94CD010C94CD010C94CD01EB
:100020000C94CD010C94CD010C94CD010C94B532FF
:100030000C94CD010C94CD010C94CD010C94CD0108
:100040000C9469320C94CD010C9483030C9413022C
:100050000C94CD010C94CD010C94CD010C94CD01E8
:100060000C94CD010C94CD01B903BB03F403F4034C
:10007000F403F403F403F403F403F403F403F403C8
:10008000C103C303C503C703C903CB03CD03CF0318
:10009000F403D303D503D703D903DB03DD03F40350
:1000A000DF03E608EC08EF08F208F708FF08070985
:1000B000A209A209A2091409170920092909A209FC
:1000C000A209A209A209A209A20935093F094B09FF
:1000D000530956095F0968096E09A209A20977093F
:1000E00080098B09BC0B4F174F17C60BD10BDC0BCC
:1000F000E70B4F17EB0B4F17F90B4F17030C0D0CBA
:10010000170C4F174F174F17270C340C410C084A88
:10011000D73B3BCE016E84BCBFFDC12F3D6C74311B
:100120009ABD56833DDA3D00C77F11BED9E4BB4C72
:100130003E916BAAAABE000000803F05A84CCDB23C
:10014000D44EB93836A9020C50B9918688083CA61D
:10015000AAAA2ABE000000803F000D0A4772626C06
:1001600020312E3167205B27242720666F7220689C
:10017000656C705D0D0A00244E005B4F50543A00D0
:100180005B5645523A312E31672E3230313831319B
:1001900031323A005B544C4F3A005B4739323A00F7
:1001A0003330003238005B4700204700204D0020EC
:1001B000530020460020540033382E005B47433A5A
:1001C00047005B484C503A24242024232024472015
:1001D000244920244E2024783D76616C20244E78DA
:1001E0003D6C696E6520244A3D6C696E6520245320
:1001F0004C50202443202458202448207E202120B5
:100200003F206374726C2D785D0D0A00536C656538
:1002100070696E6700526573746F72696E672073E0
:1002200070696E646C6500526573746F72696E6795
:100230002064656661756C74730050676D20456E4F
:100240006400436865636B204C696D697473004397
:100250006865636B20446F6F720044697361626C00
:10026000656400456E61626C656400436175746924
:100270006F6E3A20556E6C6F636B6564002724487F
:10028000277C2724582720746F20756E6C6F636B52
:1002900000526573657420746F20636F6E74696EAD
:1002A0007565005B4D53473A00414C41524D3A0051
:1002B0007C413A007C4F763A007C57434F3A007CB1
:1002C000506E3A007C46533A007C42663A007C57B6
:1002D000506F733A007C4D506F733A00536C6565F4
:1002E0007000446F6F723A00436865636B00416C45
:1002F00061726D00486F6D65004A6F6700486F6CF2
:10030000643A0052756E0049646C650000007A43DF
:1003100000007A4300007A430000FA430000FA43E9
:100320000000FA4300A00C4700A00C4700A00C47B7
:10033000000048C3000048C3000048C30A0000FF93
:10034000010AD7233C6F12033B00007A44000000EF
:100350000004000000C8410000FA43FA00000080D9
:100360003F0D0A005B5052423A006572726F723A5A
:10037000006F6B0D0A0011241FBECFEFD8E0DEBF67
:10038000CDBF27E0A0E0B1E001C01D92A136B207C9
:10039000E1F70E9468040C94993A0C940000CF9302
:1003A000DF93239AC0EBD0E083E0888384E08093DE
:1003B000B100259A20915C0230915D0240915E026D
:1003C00050915F02609158027091590280915A02D7
:1003D00090915B020E94C9359B01AC0160E070E026
:1003E0008EE793E40E94C936609300017093010187
:1003F000809302019093030188818F778883DF9136
:10040000CF9108950E94F21C0E94D81B80910B028C
:10041000811108C00E948F1D892BB1F780910A02BB
:10042000883091F308951F920F920FB60F92112406
:100430008F939F93EF93FF9380916E01E82FF0E0ED
:10044000EB5FFE4F90819093C6008F5F893609F471
:1004500080E080936E0190910401891305C0809122
:10046000C1008F7D8093C100FF91EF919F918F918B
:100470000F900FBE0F901F901895E091040191E02E
:100480009E0F993631F490E004C020910D0724FDB1
:100490000FC020916E012917C1F3F0E0EB5FFE4F12
:1004A0008083909304018091C10080628093C10099
:1004B000089590910B02911107C086FF02C0439AE4
:1004C00001C043981092150208954F925F926F9267
:1004D0007F928F929F92AF92BF92CF92DF92EF92D4
:1004E000FF926B017C0180905C0290905D02A09075
:1004F0005E02B0905F0240905802509059026090A6
:100500005A0270905B02A3019201C501B4010E94DE
:10051000E13887FF19C06091130270E080E090E03D
:100520000E9473372AE037ED43E25CE30E942139F1
:10053000A70196010E9421396B017C01A301920160
:100540000E94E13887FD0AC04092170250921802BB
:100550006092190270921A028FEF47C0A5019401B0
:10056000C701B6010E94BF361816E4F020E030E063
:10057000A901C701B6010E94BF36811109C01092BE
:100580001702109218021092190210921A022DC02E
:100590008092170290921802A0921902B0921A0249
:1005A00081E023C0C0921702D0921802E092190293
:1005B000F0921A02A5019401C701B6010E94C93543
:1005C00020910001309101014091020150910301FD
:1005D0000E9421390E94AE3720E030E040E85FE31E
:1005E0000E94CA350E944237862FFF90EF90DF901D
:1005F000CF90BF90AF909F908F907F906F905F90C3
:100600004F9008958093B300811104C08091B00091
:100610008F7703C08091B00080688093B000089508
:1006200090910B02911126C081110EC010921702F9
:10063000109218021092190210921A028091B000C2
:100640008F778093B00014C0803111F42D9801C0D1
:100650002D9A9091600291FF05C0803219F440E01C
:1006600050E0BA01CB01BA010E9465020E94020368
:10067000109215020895CF92DF92EF92FF92CF93DE
:1006800090910A02923079F06A017B01C82F0E9492
:100690000202B701A6018C2FCF91FF90EF90DF905F
:1006A000CF900C941003CF91FF90EF90DF90CF90FC
:1006B000089561EF71E088E892E00C948A2B8091B4
:1006C0000D0784FD1FC080E10E94462B8091B00081
:1006D0008F778093B000439890910A02892F8C7293
:1006E00021F480910E02867069F0943031F480918B
:1006F0000E07811105C086E001C083E00E94362B01
:100700000C947F3208951F920F920FB60F9211240E
:100710002F933F934F935F936F937F938F939F9309
:10072000AF93BF93EF93FF93E091C600E13271F076
:1007300028F4E83179F40E945F0356C0EF3321F0CA
:10074000EE3741F482E003C081E001C088E00E94FE
:10075000462B4AC0E7FF37C08E2F90E0FC01E458DB
:10076000F109ED31F10508F03FC0EC5CFF4F0C944E
:100770006C3A80E2ECCF80910A0285FF35C080E4BC
:10078000E6CF81E00DC082E00BC084E009C088E0C4
:1007900007C080E105C080E203C080E401C080E8BA
:1007A0000E942D2B21C081E00BC082E009C084E0B3
:1007B00007C088E005C080E103C080E201C080E49A
:1007C0000E94242B11C0A091EA0281E08A0F813897
:1007D00009F480E09091EB02891731F0B0E0A15963
:1007E000BE4FEC938093EA02FF91EF91BF91AF91DE
:1007F0009F918F917F916F915F914F913F912F9139
:100800000F900FBE0F901F901895FF920F931F939C
:10081000CF93DF938C01EB018091600285FF26C0AE
:10082000F0900A0280E2F81629F1C8010E944F2BCD
:100830008823E1F081E080930D0288E0F81641F012
:100840000E945F0382E00E94362B0E94D81B0EC0DC
:1008500088E00E94462B0E94D81B80910B028111D8
:1008600005C080910A028111F6CFEACF80910A0279
:10087000823041F10E94D81B80910B02811122C06D
:100880009091CA038091C903981303C00E94F21C7F
:10089000F1CFBE01C8010E940228811113C08091CE
:1008A000600281FF0FC0888584FF0CC04C815D8190
:1008B0006E817F8180E1DF91CF911F910F91FF9039
:1008C0000C943B03DF91CF911F910F91FF900895FE
:1008D000CF93DF93CDB7DEB761970FB6F894DEBF45
:1008E0000FBECDBF8091C00082608093C000109287
:1008F000C50080E18093C4008091C1008869809325
:10090000C10080E090E00E946B1E8A3009F055C55E
:1009100045E550E061E070E08BE192E00E94731EDB
:10092000892B09F44AC58AB18C618AB9209A8AB1A7
:10093000806E8AB9809181008F7E80938100809142
:100940008100886080938100809180008C7F8093FB
:100950008000809180008F708093800080916E0075
:10096000887F80936E0014BC15BC80916E008160FE
:1009700080936E0087B1887F87B988B1876088B916
:1009800080916C00876080936C0080916800826029
:10099000809368008CE0E1EFF1E0DF011D928A9521
:1009A000E9F7789410920A028091600284FF03C0F4
:1009B00081E080930A02BAE02B2EB2E03B2E99240C
:1009C000939480910A0291E1F10111929A95E9F7CD
:1009D00080930A0284E6809311028093120280932E
:1009E00013028CE0ADEFB1E01D928A95E9F7109209
:1009F000090210920D0710920E0710920F07109225
:100A000010078091EA028093EB0280E4E0E7F2E0D5
:100A100011928A95E9F764E972E080E00E94B71EBE
:100A2000811103C087E00E94392D0E94CF013B9ABB
:100A300043980E943A313D98459A80E00E941A2CD2
:100A40000E949F1D0E94C22A0E943D320E945903AB
:100A50008AE591E00E94262D8091600283FF10C0FC
:100A60000E941F2F882361F090920A0283EA92E08D
:100A70000E94262D82E492E00E94262D0E94C12E23
:100A800080910A02817899F083EA92E00E94262DF3
:100A90008DE792E00E94262D0E94C12E90920A02BC
:100AA00010E000E0F2E0EF2EA4E08A2E34C01092B5
:100AB0000A020E94CB2B80FF07C080910D07806245
:100AC00080930D070E94D81B0E944D2DE9CFE92F7E
:100AD000F0E0E159FE4F80819F5F913809F490E08A
:100AE0009093EB028F3FE9F08A3021F50E94D81BEA
:100AF00080910B02811165CFE12FF0E0EF5EF84F9E
:100B00001082F02FF170FF2E00FF18C08BE00E94C2
:100B1000392D10E000E09091EB028091EA029813E9
:100B2000D6CF0E94F21C0E94D81B80910B02882312
:100B300091F347CF8D3009F01AC4D8CF80911107B7
:100B4000882309F411C4843209F006C4998A80917B
:100B50001207833409F134F4882361F0843209F0F8
:100B600010C11AC08A3459F08835B1F0873409F0C1
:100B700008C112C082EC91E00E94262DEBC3809147
:100B80000A028F7D09F0D6C3809113078D3309F0D7
:100B9000D9C30E94E609D1C3909113079111D2C322
:100BA000833409F4B2C01CF4843239F0D3C38734DF
:100BB00069F0883509F4C9C0CDC380910A028871F3
:100BC000F82E09F0B7C30E94AF2DC4C38CEB91E09F
:100BD0000E94262D809170028C3838F088EB91E0CD
:100BE0000E94262D809170028A580E94002D89EA69
:100BF00091E00E94262D809176028A5C0E94002D51
:100C000089EA91E00E94262D809174028F5E0E94F5
:100C1000002D89EA91E00E94262D8091720225E143
:100C2000281B822F0E94002D89EA91E00E94262D28
:100C300080917302865A0E94002D89EA91E00E94F9
:100C4000262D809171029EE5981B892F0E94002D10
:100C500080917702882399F08CEA91E00E94262DFA
:100C600080917702833029F08E3139F0823039F467
:100C700004C080E30E943D0202C00E94002D8CEA65
:100C800091E00E94262D80917902803131F08032EE
:100C900031F0811107C085E303C083E301C084E321
:100CA0000E943D028CEA91E00E94262D80917802FC
:100CB000882311F088E301C089E30E943D0285EB9F
:100CC00091E00E94262D809183020E94002D82EBEC
:100CD00091E00E94262D60917F02709180028091A8
:100CE0008102909182020E94C92C8FEA91E00E94B9
:100CF000262D60917B0270917C0280917D02909103
:100D00007E0240E00E942C2C0EC080910A028230AC
:100D100069F40E945F0383EA92E00E94262D8AE52F
:100D200092E00E94262D0E94C12E14C3811102C39D
:100D3000E0920A0283EA92E00E94262D83E692E086
:100D40000E94262D0E94C12E45C080910A0281304A
:100D500009F000C30E94CB2BA82FA170FA2E80FFB0
:100D600003C0EDE0FE2EF6C283EA92E00E94262D3B
:100D70008BE692E00E94262D0E94C12E10920A025C
:100D8000E9C290910A02923008F0D4C2893409F481
:100D9000A3C034F4833271F0883409F45AC048C1D6
:100DA000823509F4EFC0833509F484C08E3409F02C
:100DB0003FC118C1809113078111C4C210E0BE0168
:100DC0006F5F7F4F812F0E94B71E811105C087E0A2
:100DD0000E94392DF12CBEC286EA91E00E94262D98
:100DE000163029F0173041F480EA91E002C083EA1E
:100DF00091E00E94262D04C086E3810F0E94002D01
:100E00008AE30E943D02CE0101960E94E72C0E94D7
:100E1000C12E1F5F183099F68AE991E00E94262DB5
:100E200080EA92E00E94E72C0E94C12E84E991E0C2
:100E30000E94262D6091AC027091AD028091AE02AD
:100E40009091AF020E94D82C0E94C12E0E94C62E03
:100E500081C28091600284FF6AC20E94CB2B80FD18
:100E600080CF80920A028091130781116BC20E9489
:100E70002F3181E00E94342F82E00E94342F0E94A3
:100E8000D81B80910B02811106C00E9459030E9459
:100E90003D320E943A3180910B0281115BC2109267
:100EA0000A020E947F3280911307811153C20E946F
:100EB0004D2D90CF809113078C3409F043C280915F
:100EC0001407803509F03EC28091150781113AC29E
:100ED00080E80E94462B3EC2E98A80911307811167
:100EE00033C040E550E06EEA73E081E197E00E9494
:100EF000731E892B51F41092110740E550E061E117
:100F000077E08EEA93E00E94B01D80E891E00E94B5
:100F1000262D0E94F52A0E94C12E8AE791E00E94A8
:100F2000262D86E50E943D028BE20E943D028CE266
:100F30000E943D028FE00E94002D8CE20E943D0243
:100F400080E80E94002DEFCEB3E0B98B8D3309F01D
:100F5000F9C183E0282F30E0F901EF5EF84F90816E
:100F6000D901A25FB84F9C938F5F90819111F2CF0E
:100F7000898B40E550E061E177E08EEA93E00E94E2
:100F8000B01DE8C180911307833509F0DBC1809162
:100F90001407843509F0D6C1809115078D3309F007
:100FA000D1C1809117078111CDC18091160784327C
:100FB00039F08A3239F0833209F0C4C182E003C0CB
:100FC00081E001C08FEF0E940E1E83EA92E00E9432
:100FD000262D87E292E00E94262D0E94C12E0E94BB
:100FE0005F03B8C1E98A8091130781111DC010E029
:100FF000812F0E94022B811104C087E00E94392DAD
:101000000EC087E791E00E94262D812F0E94002DBF
:101010008DE30E943D020E94F52A0E94352D1F5F3C
:10102000123009F497C1E4CF911184C111E001C0DD
:1010300010E0BE01635F7F4FCE0141960E941535DF
:10104000811103C072E0F72E85C1E98981E08E0F1E
:10105000898BF0E0EF5EF84F90819D3309F072C10B
:10106000112371F1482F50E0282F30E0F901EF5E95
:10107000F84F9081241B350BD901AF5EB84F9C937C
:101080008F5F90819111F0CF898B0E94E6098111C9
:1010900054C16D857E858F8598890E94043A0E948F
:1010A0004237162F0E940202E1E51E9FC001112463
:1010B00040E550E061E177E09D5F0E94B01D8ACE7F
:1010C000BE016F5F7F4FCE0141960E941535882388
:1010D00009F4B8CFE989F0E0EF5EF84F8081811123
:1010E00031C1AD84BE84CF84D88820E030E04FE7A2
:1010F00053E4C601B5010E94E13818160CF422C170
:1011000049805A806B807C80C601B5010E944237BD
:10111000062F20E030E0A901C301B2010E94BF36D2
:1011200087FD0DC1043608F441C0045680E0033049
:10113000A0F510E0000F111F000F111F823079F091
:10114000F801833019F1813019F0E55EFD4F02C0DE
:10115000E95DFD4F4082518262827382E5C00D5C81
:101160001D4F20E030E040E752E4C301B2010E948D
:10117000213920E030E040E752E40E942139D801D3
:101180006D937D938D939C931397CEC0E15CFD4F3F
:1011900077FA709477F87094DDCF8F5F0A3008F497
:1011A000D1C0843009F4CEC00A50C1CFC301B2010E
:1011B0000E94043A0E94423710E00132110508F003
:1011C000C1C0F801EF5AFF4F0C946C3A633008F439
:1011D000BCC060934B02A8C060934E02A5C0609350
:1011E0004C0202C060934D020E944E329DC080911D
:1011F0006002662311F0846095C08B7F93C080915C
:101200006002662311F080648DC08F7B8BC080915B
:101210006002662311F0806801C08F7780936002BE
:1012200080E00E941A2C80C060934F027DC04092E3
:10123000500250925102609252027092530274C056
:101240004092540250925502609256027092570298
:101250006BC080916002662311F0816001C08E7FB7
:10126000809360020E94C62B5FC08091600266235B
:1012700021F084FF6DC0806255C08F7D53C0809186
:101280006002662311F0886001C0877F809360024E
:101290000E943A3149C080916002662311F080615A
:1012A00041C08F7C3FC0609361023EC040926202A9
:1012B00050926302609264027092650235C040925F
:1012C00066025092670260926802709269022CC0B6
:1012D00070E070936B0260936A0226C040926C02C9
:1012E00050926D0260926E0270926F021DC0409229
:1012F00058025092590260925A0270925B0208C0E2
:1013000040925C0250925D0260925E0270925F02B7
:101310000E94CF0109C080916002662311F08260B3
:1013200001C08D7F809360020E94ED1D13C055E0C7
:10133000F52E10C048E0F42E0DC0F82E0BC034E09E
:10134000F32E08C023E0F22E05C096E0F92E02C06D
:101350008AE0F82E8F2D08C080910A02817211F068
:1013600089E0D5CB0E94E6090E94452DD2CB00230F
:1013700029F0893209F0CFCB0D7FCDCB813208F433
:10138000CACB8F3209F4C7CB883289F08B3389F00E
:101390001F3488F4212F30E01F5F9FE9980FF90177
:1013A000EF5EF84F9A3108F480528083B4CB02E0AC
:1013B000B2CB04E0B0CB01E0AECB87E00E94392D88
:1013C0008FEF0E940E1E0E94AF2DADCA2F923F924A
:1013D0004F925F926F927F928F929F92AF92BF9245
:1013E000CF92DF92EF92FF920F931F93CF93DF93F1
:1013F000CDB7DEB7CA54D1090FB6F894DEBF0FBE21
:10140000CDBF8AE3E0EBF2E0DF011D928A95E9F7B8
:101410008BE0E0E7F2E0A1EBB2E001900D928A955B
:10142000E1F780911107843211F00C94701781E07C
:101430008093B1021092B20283E08A8FB1E0BBA325
:10144000212C312C1CA61BA610E01B8E1F8EEE2417
:10145000E394F12CEAE0AE2EB12CF1E68F2EF3E00E
:101460009F2E8A8DE82FF0E0EF5EF84FD080DD20D0
:1014700009F437C29FEB9D0D9A3110F00C943F1781
:101480008F5F8A8FBE016A5E7F4FCE014A960E94AF
:101490001535882311F40C9441174E885F88688CA9
:1014A000798CC301B2010E94043A0E944237062F90
:1014B00070E080E090E00E9473379B01AC01C301B3
:1014C000B2010E94C93520E030E048EC52E40E94AD
:1014D00021390E948E390E944237CB01E7E4DE16A3
:1014E00029F0FDE4DF1609F4EAC035C1083209F439
:1014F000C6C020F5043168F4013108F08AC0043018
:1015000009F452C008F464C00A3009F445C00C94D0
:101510004F170C3109F440C050F4063110F00C9410
:101520004F1725E1201B2093B30226E0ADC00E31FA
:1015300099F1063209F44CC00C944F170D3309F49D
:1015400098C0A8F4053381F140F40B3209F47AC055
:10155000013309F477C00C944F170C3310F00C943E
:101560004F176AEC600F6093B70229E08DC00C350D
:1015700038F40A3508F053C0003581F10C944F1748
:101580000C3551F00F3510F00C944F172EE5201B41
:101590002093B20225E078C0009731F42F8D2111FD
:1015A0000C94431731E03F8F0093B002202F2D7F22
:1015B0002C3119F00C3509F064C0009721F00A971E
:1015C00011F00C944F17600F6093B00220E061C0DF
:1015D0004F8D41110C944317A2E0AF8F0093B102DD
:1015E000063209F050C08431910559F08E319105D1
:1015F00041F08832910529F08233910511F00C9465
:101600004F17B5010E94363A66576093B10221E048
:1016100040C06FEE600F6093B50222E035C0892BA9
:1016200031F466EA600F6093B40223E032C06A309E
:10163000710511F00C944F170A3511F40C944F17E3
:1016400024E027C0BF8DB1110C944317013331F44E
:101650001092B60228E0E3E0EF8F1BC00A9711F06A
:101660000C944F17F1E0F093B60228E033E03F8F7F
:1016700010C0892B11F00C944F172AE00AC027E004
:1016800003C020E001C021E0892B19F087E10C9410
:101690007717C70102C0880F991F2A95E2F72BA57B
:1016A0003CA528233923232B19F085E10C947717C7
:1016B000ABA5BCA5A82BB92BBCA7ABA7D2CE892BB9
:1016C00029F7063018F4033058F016C0083010F42B
:1016D0000C944F170A30F0F00E3159F00C944F175C
:1016E000002319F0013011F104C0B3E0B093B80247
:1016F0001DC00093B8021AC0043021F0053031F04B
:1017000080E101C080E28093BA0202C01092BA0266
:101710008CE00DC0093031F08091B9028064809373
:10172000B90202C01092B9028DE001C08BE0F7014E
:1017300002C0EE0FFF1F8A95E2F72BA53CA52E23D2
:101740003F23232B09F0B1CF2BA53CA52E2B3F2BFC
:101750003CA72BA786CE8D2DDD0C990BAA0BBB0BBE
:10176000FC01E654F109E531F10510F00C944F1736
:10177000EE58FF4F0C946C3A4092BC025092BD025E
:101780006092BE027092BF0280E087C04092C002A9
:101790005092C1026092C2027092C302116081E055
:1017A0007CC04092C4025092C5026092C602709200
:1017B000C702126082E071C04092C8025092C90212
:1017C0006092CA027092CB02146083E066C00093FC
:1017D000CC0284E062C0C301B2010E943B37609337
:1017E000CD027093CE028093CF029093D00285E019
:1017F00054C04092D1025092D2026092D3027092B1
:10180000D40286E04AC04092D5025092D60260923D
:10181000D7027092D80287E040C04092D90250921D
:10182000DA026092DB027092DC0288E036C020E0CF
:1018300030E04FE753E4C301B2010E94E1381816CB
:1018400014F40C9445170093DD0289E026C0409201
:10185000DE025092DF026092E0027092E1023B8D64
:1018600031603B8F8AE019C04092E2025092E3025D
:101870006092E4027092E5024B8D42604B8F8BE0E8
:101880000CC04092E6025092E7026092E802709229
:10189000E9028B8D84608B8F8CE06701082E02C07B
:1018A000CC0CDD1C0A94E2F7960122213321232B74
:1018B00011F00C944717D40102C0B595A7958A95ED
:1018C000E2F7A0FF0BC020E030E0A901C301B201A4
:1018D0000E94BF3687FF02C00C9449172C283D2870
:1018E000C0CDBB8DBB2329F0EF8DE11102C0F2E02A
:1018F000FF8F25FE0FC08091CD029091CE02A09166
:10190000CF02B091D00281389649A849B10514F0B0
:101910000C944B173BA1332329F020FC02C00C94FC
:10192000551718C08091B202813071F44F8D42304A
:10193000E1F58091B1028035C1F18823B1F120FC3D
:1019400002C00C94551731C08091710281112DC0D5
:1019500020FE1BC08091B302813039F523E333E3CD
:101960004BEC51E46091BC027091BD028091BE02CB
:101970009091BF020E9421396093BC027093BD0216
:101980008093BE029093BF0210C080917F0290911D
:101990008002A0918102B09182028093BC02909358
:1019A000BD02A093BE02B093BF0230FC10C0809174
:1019B0007B0290917C02A0917D02B0917E02809387
:1019C000D9029093DA02A093DB02B093DC028091FB
:1019D000B002843039F426FC03C08CE10C947717F4
:1019E000E89426F88091B502882369F0813029F4C3
:1019F0008FAF1DAE92E09BAF0BC01FAEA2E0ADAFAC
:101A0000B1E0BBAF05C0E2E0EFAFF1E0FDAF1BAE70
:101A10008091B302813021F02F8D2330C9F52FC082
:101A200060EBC62E62E0D62EE12CF12C3B8DA32E6E
:101A3000B12CC5010E2C02C0959587950A94E2F74A
:101A400080FF12C023E333E34BEC51E4D6019E96B2
:101A50006D917D918D919C91D1970E942139F601D4
:101A600066A777A780AB91ABFFEFEF1AFF0A24E0E0
:101A7000C20ED11C33E0E316F104D9F6CDCF80912C
:101A8000B602813029F44B8D443011F00C944D177F
:101A90008CE0E4E9F2E0DE01119601900D928A9566
:101AA000E1F78BA59CA591FD08C00091B0020A301A
:101AB000C9F00C3509F4B3C01EC18091B70287305C
:101AC00018F08DE10C94771790917602891769F3DD
:101AD000BE016F5F7F4F0E94B71E882311F40C94E4
:101AE0006317E3CF9B8D911103C08AE10C947717A4
:101AF000C10180759927892B09F46FCF6091D102BC
:101B00007091D2028091D3029091D4020E94043A43
:101B10000E9442376730A8F68091CC02843141F0B0
:101B2000823011F00C944F1727FE02C00C944F170F
:101B3000AFEA2A22662319F0615069A703C0B09169
:101B4000B702B9A760EC72E089A50E94B71E88238E
:101B500011F40C9463170091CC024090AC025090A9
:101B6000AD026090AE027090AF0240EBE42E42E016
:101B7000F42E50E7A52E52E0B52EC12CD12CEB8DC2
:101B80008E2E912CC4010C2C02C0959587950A9439
:101B9000E2F780FF35C0043151F5D501D0962D9183
:101BA0003D914D915C91D39758966D917D918D911A
:101BB0009C915B970E94C935F70126A537A540A9DE
:101BC00051A90E94C935D70150966D937D938D938D
:101BD0009C935397B2E0CB1213C0A30192010E94D1
:101BE000C935F701608B718B828B938B09C0F7012C
:101BF00086A597A5A0A9B1A9808B918BA28BB38B49
:101C0000FFEFCF1ADF0A24E0E20EF11C34E0A30E4E
:101C1000B11C43E0C416D10409F0B4CF3FC18B8D91
:101C2000882309F462CF4090AC025090AD026090DE
:101C3000AE027090AF0220E7822E22E0922EDE01EB
:101C400011967D0130EBC32E32E0D32EA12CB12CA6
:101C5000E82FF0E0F8A7EFA38FA198A50A2C02C007
:101C6000959587950A94E2F780FF29C0D7012D91B9
:101C70003D914D915C91F401608D718D828D938DBC
:101C80000E94C935D6019E962D913D914D915C9152
:101C9000D1970E94C935F60166A777A780AB91ABB3
:101CA000F2E0AF1216C0A30192010E94C935D6011D
:101CB0009E966D937D938D939C93D1970AC0F4016A
:101CC00080A991A9A2A9B3A9F60186A797A7A0AB5D
:101CD000B1ABFFEFAF1ABF0A24E0820E911C34E0D3
:101CE000E30EF11C44E0C40ED11C83E0A816B1043D
:101CF00009F0B2CFD2C09F8D933069F40E3109F450
:101D000094C0053309F4C3C00C3109F0C6C060ECBF
:101D100072E086E08DC0AB8DAA2381F3B091B4024E
:101D2000BFA34090AC025090AD026090AE027090A4
:101D3000AF0280E7A82E82E0B82E90EBE92E92E069
:101D4000F92EFE0131964F01C12CD12C2A2F30E003
:101D50003AA729A789A59AA50C2C02C09595879525
:101D60000A94E2F780FD0BC0F501808D918DA28D64
:101D7000B38DF70186A797A7A0ABB1AB44C00533DD
:101D800009F441C0FFA1F1112BC0D501D0962D91CE
:101D90003D914D915C91D397F40160817181828175
:101DA00093810E94CA35D7019E962D913D914D9108
:101DB0005C91D1970E94CA35F70166A777A780ABDF
:101DC00091ABF2E0CF121FC0A30192010E94CA356D
:101DD000D7019E966D937D938D939C93D19713C05D
:101DE000F501208D318D428D538DD7019E966D91D9
:101DF0007D918D919C91D1970E94CA35F70166A77C
:101E000077A780AB91ABFFEFCF1ADF0A24E0A20ED9
:101E1000B11C34E0E30EF11C44E0840E911C83E01D
:101E2000C816D10409F096CF69CF60EC72E087E064
:101E30000E94B71E882311F40C9463179B8D911197
:101E400003C019A61F8E2AC0A0E7B2E0E0EBF2E0C3
:101E500080E090E04B8D242F30E0A901082E02C0D5
:101E6000559547950A94E2F740FD0AC058964D9162
:101E70005D916D917C915B97408B518B628B738BE5
:101E80000196149634968330910539F706C08091F7
:101E9000B102823010F00C94511719A68091B10252
:101EA0008FA3803529F49B8D91110C9453177AC21E
:101EB000AF8DA23009F076C2BFA1B11104C0EB8D85
:101EC000E11170C22AC020E030E0A9016091BC029B
:101ED0007091BD028091BE029091BF020E94BF36F8
:101EE000882309F4E2C7FFA1FC3809F445C240F495
:101EF000F230A9F0F330B1F0F13009F053C20AC06A
:101F00002FA12E3809F438C208F433C22F3809F44F
:101F100030C248C23B8D311145C21F8E43C24BA116
:101F200044604BA38B8D882309F4DFCDBBADAB2F71
:101F3000B0E0B8ABAFA7FDADEF2FF0E0FCABEBAB83
:101F400081E090E07C010BAC02C0EE0CFF1C0A9417
:101F5000E2F70DAC02C0880F991F0A94E2F7E82A55
:101F6000F92A2B8D822F90E08E219F21892B09F455
:101F70009EC7FD01EE0FFF1FEE0FFF1FE055FD4F47
:101F8000AA0FBB1FAA0FBB1FA857BD4F2D913D9194
:101F90004D915C9166A577A580A991A90E94C9354C
:101FA0002B013C01EBA9FCA9EE0FFF1FEE0FFF1F59
:101FB000E055FD4FABA9BCA9AA0FBB1FAA0FBB1FC1
:101FC000A857BD4F2D913D914D915C9166A577A588
:101FD00080A991A90E94C9354B015C01610130E8DB
:101FE000C322DD2427FEF5C0E89427F84CE050E03A
:101FF0006EED72E088E892E00E948C3A892B11F431
:1020000081E275C78091B3028130B1F423E333E3F9
:102010004BEC51E46091D5027091D6028091D702C9
:102020009091D8020E9421396093D5027093D60214
:102030008093D7029093D8028091D5029091D602D6
:10204000A091D702B091D8028FAB98AFA9AFBAAF29
:10205000A3019201C301B2010E94213927966CAFFE
:102060007DAF8EAF9FAF2797A5019401C501B40145
:102070000E9421392B966CAF7DAF8EAF9FAF2B970F
:1020800020E030E040E850E46FA978AD89AD9AAD2A
:102090000E9421392FA938AD49AD5AAD0E9421398E
:1020A00027962CAD3DAD4EAD5FAD27970E94C9354B
:1020B0002B962CAD3DAD4EAD5FAD2B970E94C93533
:1020C0006B017C0120E030E0A9010E94BF3687FD52
:1020D000F0C6C701B6010E94C0396B017C012B9686
:1020E0002CAD3DAD4EAD5FAD2B9727966CAD7DAD64
:1020F0008EAD9FAD27970E94CA350E94C0399B01C3
:10210000AC01C701B60190580E94C9366B017C0131
:102110009FA1933021F4F7FAF094F7F8F09420E0BF
:1021200030E0A9016FA978AD89AD9AAD0E94BF36A4
:1021300087FF11C0F7FAF094F7F8F0948FA998ADE3
:10214000A9ADBAADB0588093D5029093D602A093B2
:10215000D702B093D8020FA518A9000F111F000FC6
:10216000111F00541D4FA7019601C501B4010E9423
:1021700021399B01AC01C301B2010E94C93520E0A5
:1021800030E040E05FE30E942139D8016D937D93F8
:102190008D939C9313970BA91CA9000F111F000F7F
:1021A000111F00541D4FA7019601C301B2010E94E7
:1021B0002139A50194010E94CA3520E030E040E0B9
:1021C0005FE30E942139F8016083718382839383E6
:1021D000E9C0212F30E038AF2FABE222F322EF2805
:1021E00009F469C631EF23228091B302813009F4EA
:1021F0007BC0EFA5F8A9EE0FFF1FEE0FFF1FE05405
:10220000FD4FC080D180E280F380A7019601C30119
:10221000B2010E94C9352B013C01EBA9FCA9EE0FCC
:10222000FF1FEE0FFF1FE054FD4F80819181A281BF
:10223000B3818FA798ABA9ABBAAB9C01AD01C50127
:10224000B4010E94C9354B015C01A3019201C30195
:10225000B2010E9421392B013C01A5019401C50165
:10226000B4010E9421399B01AC01C301B2010E945B
:10227000CA350E94C0394B015C01A7019601C70114
:10228000B6010E9421396B017C012FA538A949A90B
:102290005AA9CA01B9010E9421399B01AC01C701A9
:1022A000B6010E94CA350E94C0396B017C0160935F
:1022B000D5027093D6028093D7029093D8029B01E7
:1022C000AC01C501B4010E94C9354B015C01E89421
:1022D000B7F82AE037ED43EA5BE3C501B4010E9499
:1022E000E13818164CF15EC000EB12E08FA998ADF2
:1022F0000C2C02C0959587950A94E2F780FF12C0D6
:1023000023E333E34BEC51E4D80150966D917D917A
:102310008D919C9153970E942139F801608B718BAC
:10232000828B938BFFEFCF1ADF0A0C5F1F4F23E0E6
:10233000C216D104D9F65DCF20E030E040E05FE383
:10234000C501B4010E94E13818160CF459CE2FE6ED
:1023500032E143E85AE3C701B6010E9421399B01EB
:10236000AC01C501B4010E94E13818160CF448CE46
:1023700019C03BA130613BA38FA18E58823018F465
:102380004BA148604BA38B8D882309F4AECB4CE066
:1023900050E06EED72E088E892E00E948C3A892B62
:1023A00009F42ECE2BA121709BA190FF03C0C10187
:1023B0008E7D03C0C1018E7D9C7FAF8DA111937E68
:1023C000892B09F07AC58E01035F1F4F89E0F80160
:1023D00011928A95E9F7222309F44BC08BA59CA59D
:1023E000867B892B09F06BC58091B002853311F093
:1023F000811165C580917B0290917C02A0917D0244
:10240000B0917E02898B9A8BAB8BBC8B90917902B9
:1024100080917802892B4091BC025091BD0260915D
:10242000BE027091BF024D875E876F87788B846094
:102430008D8B8091600285FF06C08EED92E00E9438
:102440004F2B81113EC5B8018EED92E00E9405042C
:1024500080910A02811139C50E948F1D892B09F4D0
:1024600034C580E280930A020E94D81E0E94FD3487
:102470002CC580916002F090790281FF26C08FA167
:102480008150833018F0FBA1F064FBA32B8D222335
:1024900039F03F8D323021F44BA140684BA315C079
:1024A00080E1F81212C08091700281509BA190745B
:1024B000833030F4992349F09BA190629BA305C01F
:1024C000911103C0ABA1A062ABA38091CD0290910A
:1024D000CE02A091CF02B091D0028093840290935B
:1024E0008502A0938602B09387028091B202809306
:1024F0007102882311F088E08D8B8091BC0290914D
:10250000BD02A091BE02B091BF0280937F02909362
:102510008002A0938102B09382028D879E87AF874D
:10252000B88B8090D9029090DA02A090DB02B09034
:10253000DC02A501940160917B0270917C02809184
:102540007D0290917E020E94BF36BBA1B074EB2E3B
:10255000811103C0EBA1E5FF20C0FF2071F0FBA1BA
:10256000F7FD0BC0EE2021F040E050E0BA0102C0C0
:10257000B501A4018F2D0E943B038091D902909157
:10258000DA02A091DB02B091DC0280937B0290938F
:102590007C02A0937D02B0937E02E1100CC080917A
:1025A0007B0290917C02A0917D02B0917E02898B8A
:1025B0009A8BAB8BBC8B8091DD02809383028091E0
:1025C000BA0290917902981751F049895A896B891A
:1025D0007C890E943B038091BA02809379029D8995
:1025E00080917902892B8D8BF090B90280917802CD
:1025F0008F1569F080910A02823029F00E94020250
:102600008F2D0E9459028091B902809378029D8992
:1026100080917802892B8D8B8091B002843099F45F
:10262000C090D102D090D202E090D302F090D402B8
:1026300080910A02823039F00E94020240E0C70114
:10264000B6010E940E328091B5028093740280918F
:10265000B302809372022F8D233071F58091B60200
:1026600080937502811108C01092E6021092E70271
:102670001092E8021092E902C090E602D090E702C0
:10268000E090E802F090E902A70196016091AC02A7
:102690007091AD028091AE029091AF020E94BF3660
:1026A000882351F0C092AC02D092AD02E092AE020B
:1026B000F092AF020E94C62B8091B70290917602F1
:1026C000981769F0809376028CE0FE013196A4E9B8
:1026D000B2E001900D928A95E1F70E94C62B80919D
:1026E000B402809373028091B0028632F1F138F423
:1026F0008C3109F18E31F9F08A3069F04FC08C3598
:10270000D1F1863609F441C0883209F047C068E843
:1027100072E087E02DC060EC72E089A50E94FA1D8E
:102720008091760239A5381339C08CE0E0ECF2E0F4
:10273000A4E9B2E025C08D8981608D8B4F8D442343
:1027400029F0B8018EED92E00E940504B80180ECFA
:1027500092E00E9405048CE0E0ECF2E0A8E8B2E030
:1027600001900D928A95E1F719C068E872E086E061
:102770000E94FA1D13C08CE0EEEDF2E0A0EAB2E098
:1027800001900D928A95E1F707C08CE0E0EAF2E053
:10279000DF011D928A95E9F70E94C62B8091B10254
:1027A00080937002803509F41CC3BF8DB23009F0EC
:1027B00018C3813021F4BE01635F7F4F06C08111D1
:1027C00009C08D8981608D8BB8018EED92E00E94E9
:1027D0000504FEC28250823008F093C28091D50277
:1027E0009091D602A091D702B091D8028F8F98A372
:1027F000A9A3BAA3ABAD94E0A99F70011124F7017E
:10280000E857FD4FF8A7EFA3970120543D4F3AA793
:1028100029A7D9014D905D906D907C9020813181E8
:1028200042815381C301B2010E94CA356BA77CA7C4
:102830008DA79EA7EDADB4E0EB9F80011124980118
:1028400028573D4F3CAF2BAFC80180549D4F9EAFE2
:102850008DAFDC018D909D90AD90BC90F9012081F1
:10286000318142815381C501B4010E94CA356FA7ED
:1028700078AB89AB9AAB77FA709477F87094D501FE
:10288000C401B0588B8F9C8FAD8FBE8FF701E25281
:10289000FD4F2BA53CA54DA55EA560817181828170
:1028A00093810E94C9356B017C01F801E252FD4F12
:1028B0002FA538A949A95AA9608171818281938184
:1028C0000E94C9354B015C01A7019601C301B20109
:1028D0000E9421396BAB7CAB8DAB9EABA501940103
:1028E0006B8D7C8D8D8D9E8D0E9421399B01AC015D
:1028F0006BA97CA98DA99EA90E94CA356BAB7CAB44
:102900008DAB9EABA5019401C301B2010E94213998
:102910004B015C01A70196016B8D7C8D8D8D9E8D89
:102920000E9421399B01AC01C501B4010E94C93547
:102930002BA93CA94DA95EA90E9449366B017C01D7
:102940009BA192FF13C02DEB37E346E055EBC70187
:10295000B6010E94E13887FD1DC02BED3FE049EC38
:1029600050E4C701B6010E94C93512C02DEB37E310
:1029700046E055E3C701B6010E94BF36181654F071
:102980002BED3FE049EC50E4C701B6010E94CA3587
:102990006B017C018090540290905502A0905602E9
:1029A000B09057022F8D38A149A15AA1CA01B9018F
:1029B0000E94CA35A50194010E94C935A501940160
:1029C0000E9421390E94C0394B015C0120E030E0B7
:1029D00040E05FE3C701B6010E9421392F8D38A185
:1029E00049A15AA10E9421399F77A50194010E9413
:1029F000C9360E94AE370E9442377CAB6BABDB011D
:102A0000AB2B09F4D8CE1D894B01A12CB12C13FF9F
:102A100012C0C501B4010E9471379B01AC016D85E4
:102A20007E858F8598890E9421396D877E878F8763
:102A3000988B177F1D8BC501B4010E9471374B0124
:102A40005C019B01AC01C701B6010E94C9366BA3B2
:102A50007CA38DA39EA3EFADB4E0EB9FC001112436
:102A60008C0108571D4FFC01E252FD4FD8012D91FA
:102A70003D914D915C9160817181828193810E9431
:102A8000C935A50194010E94C93627966CAF7DAF68
:102A90008EAF9FAF27972BA13CA14DA15EA1CA018C
:102AA000B9010E9421399B01AC0160E070E080E037
:102AB00090E40E94C9356B017C012BEA3AEA4AE2B4
:102AC0005EE36BA17CA18DA19EA10E9421394B01E7
:102AD0005C0120E030E040E850E4C701B6010E940C
:102AE000CA359B01AC01C501B4010E9421396FAB0D
:102AF00078AF89AF9AAF20E030E040E05FE3C701F4
:102B0000B6010E94213923966CAF7DAF8EAF9FAF87
:102B100023971F8E22242394312CEBA9FCA9E215C4
:102B2000F30509F448CEBF8DBC3008F044C02B8DAE
:102B30003C8D4D8D5E8D23966CAD7DAD8EAD9FAD84
:102B400023970E9421396B017C01A30192016FA997
:102B500078AD89AD9AAD0E942139A70196010E94F6
:102B6000CA357B016C01A301920123966CAD7DAD4A
:102B70008EAD9FAD23970E9421394B015C012B8DB7
:102B80003C8D4D8D5E8D6FA978AD89AD9AAD0E945B
:102B900021399B01AC01C501B4010E94C9352B014B
:102BA0003C01EF8DEF5FEF8F470156018B8E9C8EBE
:102BB000AD8EBE8E65C0B10180E090E00E9471379D
:102BC0002BA13CA14DA15EA10E9421396B017C018A
:102BD0000E94C4366B8F7C8F8D8F9E8FC701B6018C
:102BE0000E94B2394B015C01A9A5BAA5CD90DD9038
:102BF000ED90FC90F7FAF094F7F8F094ADADBEAD1F
:102C00008D919D910D90BC91A02D8F8F98A3A9A31C
:102C1000BAA3A70196016B8D7C8D8D8D9E8D0E9430
:102C200021392B013C012F8D38A149A15AA1C501A1
:102C3000B4010E9421399B01AC01C301B2010E9481
:102C4000CA352B013C01A7019601C501B4010E94C0
:102C500021396B017C012F8D38A149A15AA16B8DBF
:102C60007C8D8D8D9E8D0E9421399B01AC01C70109
:102C7000B6010E94C9356B8F7C8F8D8F9E8F1F8E02
:102C8000A30192016BA57CA58DA59EA50E94CA35C6
:102C9000EFA1F8A560837183828393832B8D3C8D94
:102CA0004D8D5E8D6FA578A989A99AA90E94CA3514
:102CB000ABADBCAD6D937D938D939C93139727968D
:102CC0002CAD3DAD4EAD5FAD2797F80160817181B0
:102CD000828193810E94CA35D8016D937D938D9333
:102CE0009C931397BE01635F7F4F88E892E00E9438
:102CF000050480910B0281116BC0BFEF2B1A3B0AB8
:102D00000CCF8D8984608D8B80910A02823009F40A
:102D10005FC00E94020280910B02811162C0FBA180
:102D2000F071FF2E10920F022BA123FB882780F950
:102D30000E941A2C86B180729091F001891749F097
:102D400084E00E94362B0E94D81B80E00E941A2C3F
:102D500048C0B8018EED92E00E94050481E08093A6
:102D6000090282E00E94462B0E94D81B80910B0230
:102D7000811137C080910A028111F6CF809109023A
:102D8000813081F4FF2051F08CE0E1EFF1E0ADEF14
:102D9000B1E001900D928A95E1F707C085E00E94AD
:102DA000362B03C081E080930F021092090280E06D
:102DB0000E941A2C0E94D81B0E94C22A0E949F1DAA
:102DC0000E943D320E94C62E80910F0281118CC05C
:102DD0008CE0EEEDF2E0A8E8B2E001900D928A9569
:102DE000E1F78091B80280937702882309F47FC0CD
:102DF0000E9402028091770290910A02833041F48E
:102E00009230D1F188E00E94462B0E94D81B34C03A
:102E100081E08093700210927402109273021092FB
:102E2000710210927602109279021092780284E672
:102E3000809311028093120280931302923091F0DA
:102E400064E972E080E00E94B71E8823E1F10E94ED
:102E5000C62B40E050E0BA0180E00E94100380E001
:102E60000E94590283EA92E00E94262D8AE392E0B2
:102E70000E94262D0E94C12E109277022FC081E061
:102E800036C082E034C088E132C086E230C089E1D9
:102E90002EC084E02CC08BE12AC085E228C084E1EA
:102EA00026C08EE124C08FE122C086E120C080E2EE
:102EB0001EC082E21CC083E21AC084E218C080E116
:102EC00016C08FE014C087E012C08CE0EEEDF2E097
:102ED000A8E8B2E001900D928A95E1F780E007C082
:102EE0001A8E1BA20C94200A0E9459037ACFC65B4B
:102EF000DF4F0FB6F894DEBF0FBECDBFDF91CF918D
:102F00001F910F91FF90EF90DF90CF90BF90AF9007
:102F10009F908F907F906F905F904F903F902F90F9
:102F200008953F924F925F926F927F928F929F92FD
:102F3000AF92BF92CF92DF92EF92FF920F931F93C7
:102F4000CF93DF93CDB7DEB7A4970FB6F894DEBF6B
:102F50000FBECDBF10910E07112391F181E0809338
:102F60000A0289EA92E00E94262D812F0E94002DFC
:102F70000E94352D85EF91E0019739F0EFE9FFE0F0
:102F80003197F1F700C00000F7CF1150123030F048
:102F90008FB7F89410920E078FBF12C083EA92E0A9
:102FA0000E94262D81E992E00E94262D0E94C12ECA
:102FB00080E10E943C2B80910D0784FFFCCFE8CF7D
:102FC00010910D07112309F4C0C214FF04C081E061
:102FD00080930B02D5C310FFC4C18CE0E1EFF1E098
:102FE000DE01599601900D928A95E1F7BE01675E68
:102FF0007F4FCE010D960E948A2B8CE30E943D02EA
:1030000080910A028830E1F058F4813099F1A8F0FB
:10301000823099F1843009F043C084EF92E03EC0E1
:10302000803229F118F4803171F03AC0803441F1D6
:103030008038B1F58CED92E031C087E093E02EC08E
:1030400083E093E02BC080910C0287FD10C08DEFD0
:1030500092E00E94262D80910C0280FF06C080E342
:103060001AC082FF17C085FFFACF81E314C089EF31
:1030700092E014C08EEE92E011C088EE92E00EC095
:1030800082EE92E00E94262D80910C0283FFE9CF10
:1030900083E301C082E30E943D0202C00E94262D0C
:1030A00080914F02F82FF170BF2E80FF07C08091F2
:1030B0001602882319F085ED92E053C04090AC02CF
:1030C0005090AD026090AE027090AF0254E9852E30
:1030D00052E0952E9E012F5F3F4F7901CE010D9654
:1030E0006C0100E0F40161917191819191914F0126
:1030F00020853185428553850E94CA35F70160835A
:10310000718382839383023061F4A30192010E9450
:10311000CA35F7016083718382839383BB2019F0E2
:10312000CACFB11011C0F701208131814281538192
:10313000F60160817181828193810E94C935F60117
:1031400060837183828393830F5FF4E0EF0EF11C41
:1031500024E0C20ED11C033029F6B110ACCF8EECA6
:1031600092E00E94262DCE010D960E94E72C8091C0
:103170004F0281FF1FC089EC92E00E94262D9091A2
:10318000EB068091CA03981710F0815F01C081504F
:10319000891B0E94002D8CE20E943D028091EB026F
:1031A0009091EA02981710F0805801C08150891B55
:1031B0000E94002D84EC92E00E94262D80910A024C
:1031C0008C7749F06091AF037091B0038091B103A7
:1031D0009091B20303C060E070E0CB010E94C92C63
:1031E0008CE20E943D02609117027091180280915A
:1031F000190290911A0240E00E942C2C0E941F2F6D
:10320000F82E0E94CB2B082F86B1982F90728091B8
:10321000F001E92EE8268F2D802B8E2981F18FEB8E
:1032200092E00E94262DEE2019F080E50E943D02DA
:10323000FF2079F0F0FE03C088E50E943D02F1FE18
:1032400003C089E50E943D02F2FE03C08AE50E94A8
:103250003D020023A1F000FF03C084E40E943D0270
:1032600001FF03C082E50E943D0202FF03C088E423
:103270000E943D0203FF03C083E50E943D0280914E
:103280001602882321F081508093160218C0809185
:103290000A028C7711F08DE101C089E0809316025B
:1032A00080911502811103C081E08093150289EBA2
:1032B00092E00E94262DCE0101960E94E72C0091FB
:1032C0001502002321F001500093150242C08091A5
:1032D0000A028C7711F083E101C089E08093150226
:1032E00084EB92E00E94262D809111020E94002D15
:1032F0008CE20E943D02809112020E94002D8CE21D
:103300000E943D02809113020E94002D8091B00026
:1033100087FF05C02D9B02C002E001C001E0439B76
:1033200003C040E4F42E03C0002399F0F12C80EB9D
:1033300092E00E94262D002339F0013011F483E53C
:1033400001C083E40E943D02FF2019F086E40E9440
:103350003D028EE30E943D020E94352D81E00E94D5
:103360003C2B812F887E09F467C080910A02982F38
:10337000937009F050C08872A1F080910C02807C9B
:1033800081F40E94962682E080930E0280910A02C8
:10339000803239F417FDF2C180910C02806880936D
:1033A0000C0280910A02811103C091E090930C02FB
:1033B00016FF07C085FD05C090910C0290649093A4
:1033C0000C0213FF05C0807E19F480E180930A028D
:1033D00015FF21C083EA92E00E94262D8FE492E03F
:1033E0000E94262D0E94C12E80910C0287FD0EC0E6
:1033F00090910A02903439F483FFBCC1837E8260CD
:1034000080930C02B7C1903809F0B4C180910C02CE
:10341000806280930C0217FF0CC080910A028130F9
:1034200029F480910C02856080930C0280E88093DF
:103430000A0288EE0E943C2B11FF44C0812F88763F
:10344000F1F580910A02803471F480910C0285FDBF
:103450000AC084FF03C010920A0205C082FF03C0A5
:10346000886080930C0280910A02882381F084FF97
:1034700026C090910C0290FF22C0803141F48091CF
:103480001402882321F088608093140218C01092DF
:103490000E020E948F1D892B71F080910C0286FD17
:1034A0000AC010920C0288E080930A020E94D81E83
:1034B0000E94FD3404C010920C0210920A0282E0B5
:1034C0000E943C2B12FF41C080910A02807D9091A6
:1034D0000C028823D9F080910D02811117C097FD4D
:1034E00015C00E9496268091CA038093C8030E944B
:1034F000BA2680910E0281FF05C090910C02916066
:1035000090930C02897F80930E021CC097FF0AC023
:1035100010920E020E949F1D0E94C22A0E9459030F
:103520000E943D3280910C0285FF08C08F77816038
:1035300080930C0280E480930A0204C010920C0273
:1035400010920A0284E00E943C2B90910F0799236D
:1035500009F4ABC08FB7F89410920F078FBF40915A
:10356000110290FD02C0842F01C084E691FD865FA8
:1035700092FD8A5093FD8F5F94FD8150893C08F045
:1035800088EC8A3008F48AE03091120295FD02C07E
:10359000232F01C024E696FD22E397FD29E148137D
:1035A00003C0231709F481C08093110220931202F3
:1035B000109215021091CA033090EB0689E9D82EBB
:1035C00096E7E92E26E9F22E0EE732E3432E131595
:1035D00009F457C0812E912C489CC001499C900D44
:1035E0001124FC01E553FC4F5F01CF010E941C1D1B
:1035F000562E672E782EC92E2D2D3E2D4F2D502F55
:103600000E94E13818164CF42D2D3E2D4F2D502FD1
:103610006D2D7E2D8F2D902F08C0252D362D472DF9
:103620005C2D652D762D872D9C2D0E942139F5016D
:10363000668B778B808F918F489CC001499C900D41
:1036400011249C0125533C4F7901F90182A093A0DC
:10365000A4A0B5A0A501940166897789808D918D7C
:103660000E94E13818162CF4F701868A978AA08EFA
:10367000B18E1F5F103109F410E0D52C73010C2DB1
:10368000A6CF8D2D9E2DAF2DB02F8093090790933F
:103690000A07A0930B07B0930C070E94962680910F
:1036A000CA038093C8030E94BA2610911007112301
:1036B00009F459C08FB7F894109210078FBF9091FA
:1036C000130210FD02C0892F01C084E611FD865F40
:1036D00012FD8A5013FD8F5F14FD8150893C08F064
:1036E00088EC8A3008F48AE09817D1F080931302AE
:1036F00080910A0281110DC040917B0250917C02A1
:1037000060917D0270917E02809179020E94100387
:1037100005C080910E02886080930E0210921502FF
:1037200080910A0215FF0DC0803159F49091140266
:10373000911102C092E003C090FF03C09460909387
:103740001402107C81F0882311F0887361F01091CD
:10375000780216FF02C01F7B01C01064812F0E94F7
:1037600059021093780280910A028C7F49F00E94DE
:10377000D81E06C080E480930A0248CE80E218CEAC
:10378000A4960FB6F894DEBF0FBECDBFDF91CF91E8
:103790001F910F91FF90EF90DF90CF90BF90AF906F
:1037A0009F908F907F906F905F904F903F90089583
:1037B000CF92DF92EF92FF921F93CF93DF930E94FD
:1037C000911780910C02882309F404C10E948F1D77
:1037D000009771F4C091790280917802C82BC09053
:1037E0007B02D0907C02E0907D02F0907E020EC0C1
:1037F000FC01C189C073439B02C020E401C020E0EA
:10380000C22BFC01C6A4D7A4E0A8F1A88091600255
:1038100081FF03C080E20E94242BDC2FD07311E0D3
:10382000C07C80910C02882309F4D4C090910B02D3
:103830009111D0C080FFCBC090910A02292F207C2B
:1038400009F47AC082FD12C01092140240E050E0E8
:10385000BA0180E00E94100380E00E94590280912A
:103860000C028D7F846080930C02B1C09038E1F42B
:1038700083EA92E00E94262D8CE092E00E94262DA1
:103880000E94C12E40E050E0BA0180E00E94100387
:1038900080E00E9459020E947F3280910B028111C8
:1038A00099C00E949117F9CF903449F40E94CB2B14
:1038B00080FD05C080910C028F7D80930C02809169
:1038C0000C0283FF84C0909179029923C1F081FD9D
:1038D00016C08091600281FF06C080910E02886050
:1038E00080930E020CC0B701A6018D2F0E94100319
:1038F00041E060E070E080E890E40E940E32809148
:103900007802882371F080910C0281FD0AC08C2F0F
:103910000E94590241E060E070E080E89FE30E946D
:103920000E3280910C0281FD52C0806180930C02A6
:1039300082E00E94462B4BC0809114028823C9F17B
:1039400081FF0DC0809179028823B1F040E050E002
:10395000BA0180E00E9410031093140238C08C70EA
:10396000B1F18091790281110AC08091140283FF24
:1039700003C082E00E94462B1092140228C083EA02
:1039800092E00E94262D85E192E00E94262D0E9461
:10399000C12E8091600281FF06C080910E02886076
:1039A00080930E02E2CFB701A6018D2F0E94100373
:1039B000DCCF80910E0283FF0AC0B701A6018D2FD4
:1039C0000E94100380910E02877F80930E020E9456
:1039D000911727CFDF91CF911F91FF90EF90DF904C
:1039E000CF9008950E948F1D892B19F082E00C94CE
:1039F000462B0895F894F999FECF92BD81BD81E0E0
:103A00008FBB80B58627482F082E000C550B262F1C
:103A100030E024233523232B39F06F3F19F060BDAC
:103A200084E006C084E104C0882321F060BD84E204
:103A30008FBBF99A78940895BF92CF92DF92EF925C
:103A4000FF920F931F93CF93DF937C01FC0102A59C
:103A500013A5D4A5C5A5818980FF18C06091120265
:103A600070E080E090E00E9473372AE037ED43E297
:103A70005CE30E9421399B01AC01B8018D2F9C2F82
:103A80000E9421398B01D82FC92F2DC082FD17C06C
:103A90006091110270E080E090E00E9473372AE0AC
:103AA00037ED43E25CE30E9421399B01AC01B80190
:103AB0008D2F9C2F0E9421398B01D82FC92FF70100
:103AC000B6A0C7A0D0A4F1A42B2D3C2D4D2D5F2D69
:103AD000B8018D2F9C2F0E94E138181624F40B2D6D
:103AE0001C2DDD2DCF2D20E030E040E85FE3B80154
:103AF0008D2F9C2F0E94E138181624F000E010E072
:103B0000D0E8CFE3B8018D2F9C2FDF91CF911F918B
:103B10000F91FF90EF90DF90CF90BF90089580912C
:103B2000CA039091EB06981739F022E3829FC001F7
:103B3000112485539C4F089580E090E008958CE116
:103B4000E1EFF6E0DF011D928A95E9F71092CA03D2
:103B50001092EB0681E08093C9031092C803089588
:103B60009F92AF92BF92CF92DF92EF92FF920F930C
:103B70001F93CF93DF935C018A017B01E40EF51E56
:103B8000EB01912C6C01C61AD70ACE018C0D9D1D3C
:103B9000CE15DF0589F0911008C0292D990C330B43
:103BA000232F221F2227221F01C021E06991922E7C
:103BB000960E0E94FA1CE9CF692DC501800F911F56
:103BC000DF91CF911F910F91FF90EF90DF90CF90F9
:103BD000BF90AF909F900C94FA1C6AE080E090E058
:103BE0000E94FA1C45E550E06BE172E081E090E054
:103BF0000C94B01D0F931F93CF93C82F8B010E947D
:103C000002022DE0C29FC00111244CE050E0B80137
:103C10009E5FCF911F910F910C94B01DEF92FF9278
:103C20000F931F93CF93DF93CDB7DEB72C970FB6CB
:103C3000F894DEBF0FBECDBF182F80FF0BC085E507
:103C4000ECE0F3E0ABE1B2E005900D928A95E1F78C
:103C50000E94ED1D11FF10C0CE0101967C018CE089
:103C6000F70111928A95E9F700E0B701802F0E94D1
:103C7000FA1D0F5F0830C9F712FF14C060E080E042
:103C800093E00E94FA1C60E081E093E00E94FA1C3D
:103C900060E081E593E00E94FA1C60E082E593E039
:103CA0000E94FA1C13FF0AC060E08EEA93E00E94B3
:103CB000FA1C60E08FEA93E00E94FA1C2C960FB683
:103CC000F894DEBF0FBECDBFDF91CF911F910F9152
:103CD000FF90EF900895F999FECF92BD81BD81E0EC
:103CE0008FBB80B508959F92AF92BF92CF92DF9223
:103CF000EF92FF920F931F93CF93DF935B018A01A3
:103D00007C01E40EF51EEC01912C6B01C81AD90A56
:103D1000C6018C0F9D1FCE15DF0589F00E946B1E1A
:103D2000911008C0292D990C330B232F221F222715
:103D3000221F01C021E0982E920E8993E9CFC50180
:103D4000800F911F0E946B1E21E030E0981611F049
:103D500020E030E0C901DF91CF911F910F91FF90DA
:103D6000EF90DF90CF90BF90AF909F9008951F93FA
:103D7000CF93DF93182FEB018DE0189FB001112432
:103D80007E5F4CE050E0CE010E94731E892B59F4F7
:103D90008CE0FE0111928A95E9F7BE01812F0E9405
:103DA000FA1D80E001C081E0DF91CF911F9108955D
:103DB0002F923F924F925F926F927F928F929F923B
:103DC000AF92BF92CF92DF92EF92FF920F931F9329
:103DD000CF93DF93CDB7DEB7EC970FB6F894DEBF85
:103DE0000FBECDBF80910E0280FD87C79091120358
:103DF0008091EC06981709F480C78091EF069091A6
:103E0000F006892B09F015C310910E0212FF09C0AC
:103E10008091EB0622E3289FC001112485539C4F1B
:103E200002C00E948F1D9093F0068093EF062090B1
:103E3000EF063090F0062114310409F45EC70091BA
:103E40009903802F817000FF03C010929903EAC08C
:103E5000909198039F5F953009F0892F8093980384
:103E6000E82EF12C32E13E9DF0013F9DF00D112432
:103E7000E25CFC4FF093EE06E093ED06D101509624
:103E80009C915097908BE2E18E9FC001112420E01D
:103E900030E04D915D916D917D91F901E80FF91F31
:103EA000E25CFC4F689412F8440F551F661F771FA1
:103EB0001694D1F740835183628373832C5F3F4F05
:103EC0002C30310531F722E12E9DF0012F9DF00DB0
:103ED00011249F01225C3C4FF10184859585A685C4
:103EE000B78543E0880F991FAA1FBB1F4A95D1F7DA
:103EF000F90184879587A687B787D1011C966D91B4
:103F00007D918D919C911F970E94713760939E03C4
:103F100070939F038093A0039093A103F101268DDA
:103F2000378D40A151A10E94C9369B01AC0160931D
:103F3000A2037093A3038093A4039093A50360E06E
:103F400070E080EA9FE30E94C9366093A6037093F5
:103F5000A7038093A8039093A90310929A03109249
:103F60009B0310929C0310929D0311FD02C003FF5E
:103F70001FC06091B7037091B8038091B90390910D
:103F8000BA036093AF037093B0038093B10390932F
:103F9000B2039B01AC010E942139D10152966D936D
:103FA0007D938D939C935597077F009399030FC042
:103FB000F10162897389848995890E94C03960936F
:103FC000AF037093B0038093B1039093B203F2E117
:103FD000FE9DC001FF9D900D11249C01225C3C4F71
:103FE0007901D90151961C928091600281FF1AC01B
:103FF000F101818985FF16C022A533A544A555A5E9
:1040000060E070E080E89FE30E94C9366093C303DC
:104010007093C4038093C5039093C603E1E0D70176
:104020005196EC931092AB031092AC031092AD0337
:104030001092AE03D1015A962D913D914D915C9114
:104040005D9729833A834B835C8360E070E080E076
:104050009FE30E94C9364B015C01F101468C578CED
:1040600060A071A011FF4BC0F2E0F093AA03D10150
:104070005296CD90DD90ED90FC905597A70196015A
:104080000E9421399B01AC01C301B2010E94C935D4
:104090004B015C0120E030E0A9010E94BF3687FFA0
:1040A0001DC029813A814B815C81CA01B9010E94FE
:1040B000CA35A30192010E9421399B01AC01C701BD
:1040C000B6010E94C9350E94C0396093B70370934E
:1040D000B8038093B9039093BA03A8C18092AB034D
:1040E0009092AC03A092AD03B092AE031092B703CE
:1040F0001092B8031092B9031092BA0397C11092AC
:10410000AA034092BB035092BC036092BD0370921D
:10411000BE0312FF0CC01092B7031092B8031092A6
:10412000B9031092BA03C12CD12C760124C0E091BE
:10413000CA03EF5FE03109F4E0E08091EB068E17EF
:1041400059F0B2E3BE9FF0011124E553FC4FC28841
:10415000D388E488F58803C0C12CD12C7601C7012F
:10416000B6010E94C0396093B7037093B80380937F
:10417000B9039093BA03C1010E941C1D698B7A8B0D
:104180008B8B9C8B9B01AC010E94213969877A87BC
:104190008B879C87D10152962D913D914D915C91D9
:1041A00055972D833E834F8358870E94BF3687FFE4
:1041B0006CC029853A854B855C856D817E818F81B8
:1041C00098850E94C935A50194010E9421399B015F
:1041D000AC01C301B2010E94C9356093BB03709367
:1041E000BC038093BD039093BE0320E030E0A9019F
:1041F0000E94BF3618163CF1B2E0B093AA032981A1
:104200003A814B815C81CA01B9010E94CA35A30180
:1042100092010E9421399B01AC016D817E818F81C9
:1042200098850E94C9350E94C0396093B703709386
:10423000B8038093B9039093BA038091990388607F
:1042400080939903F3C0A701960169857A858B85D0
:104250009C850E94C935A50194010E942139609373
:10426000BF037093C0038093C1039093C203298955
:104270003A894B895C892093B3033093B40340930C
:10428000B5035093B60333E0B6C0A70196016D8124
:104290007E818F8198850E94C935A50194010E9475
:1042A0002139A30192010E94CA3520E030E040E0AC
:1042B0005FE30E9421396D877E878F87988B20E08E
:1042C00030E0A9010E94E13818160CF097C02D8546
:1042D0003E854F855889C301B2010E94E138181606
:1042E0000CF088C0A701960169857A858B859C852D
:1042F0000E94C935A50194010E9421399B01AC019E
:104300006093BF037093C0038093C1039093C20373
:104310006D857E858F8598890E94E1381816CCF5C9
:1043200089899A89AB89BC898093B3039093B4033C
:10433000A093B503B093B6032D813E814F8158857C
:1043400069857A858B859C850E94BF36811104C062
:1043500091E09093AA036AC02D813E814F815885D8
:1043600069857A858B859C850E94C935A501940154
:104370000E9421399B01AC01C301B2010E94C935E1
:104380006093BB037093BC038093BD039093BE0303
:104390004DC02D853E854F8558892093BB033093B2
:1043A000BC034093BD035093BE032093BF033093DF
:1043B000C0034093C1035093C20329813A814B81CA
:1043C0005C81CA01B9010E94CA352D853E854F85A1
:1043D00058890E942139A70196010E94CA350E947E
:1043E000C0396093B3037093B4038093B503909383
:1043F000B6031CC032E03093AA0318C01092BB036E
:104400001092BC031092BD031092BE038091B703BB
:104410009091B803A091B903B091BA038093B3030C
:104420009093B403A093B503B093B60318601093B0
:104430000E0280913D03482F50E05A8B498B87E054
:10444000849FF001859FF00D1124ED5EFC4F80915B
:1044500098038483A091EF06B091F006BCAFABAF98
:104460005E96BC91BAA3EBADFCADF78DFBA3ABADF3
:10447000BCAD9096BC91BCA3EBADFCADF1A1FDA38E
:104480002091A6033091A7034091A8035091A9035E
:104490006AA17BA18B2F9F2F0E94C9356EA77FA792
:1044A00088AB99AB20E030E0A9010E94BF3687FFBE
:1044B00004C01EA61FA618AA19AA2091B3032E8B0A
:1044C0003091B4033F8B4091B503488F5091B603B0
:1044D000598F8091BB038A8F9091BC039B8FA091D1
:1044E000BD03AC8FB091BE03BD8FE091AF03E983F4
:1044F000F091B003FD832091B10329873091B2037D
:104500003D874091BF034EA35091C0035FA38091AC
:10451000C10388A79091C20399A7A091AA03AD8B6C
:10452000B091AB03BAA7E091AC03EBA7F091AD0358
:10453000FCA72091AE032DA73091B7033BAB409170
:10454000B8034CAB5091B9035DAB8091BA038EAB0D
:104550002EA13FA148A5592F6A8D7B8D8C8D9D8DF5
:104560000E94BF36811103C092E09AAB02C0A1E065
:10457000AAAB3AA02BA01CA10DA18EE3C82E83EC00
:10458000D82E8EE2E82E89E3F82E412C512C3201F0
:10459000CE8EDF8EE8A2F9A23D89313009F4F2C057
:1045A000ABADBCAD313008F47BC0333009F020C175
:1045B0005A962D913D914D915C915D97C701B60141
:1045C0000E9421394B015C012E893F89488D598D0C
:1045D00069817D8189859D850E94C9359B01AC01DA
:1045E000C501B4010E94E13887FD31C02A8D3B8DA1
:1045F0004C8D5D8D6AA17BA18CA19DA10E94C935C6
:104600009B01AC010E94CA356B017C0129813D816F
:1046100049855D856E897F89888D998D0E94CA350F
:104620009B01AC01C701B6010E94C9366B017C0138
:10463000BE89B983EF89ED83F88DF987298D2D87A0
:104640003A8C2B8C1C8D0D8D31E03D8B51C120E0BF
:1046500030E040E05FE3C501B4010E9421399B01D5
:10466000AC0169817D8189859D850E94C935A7013D
:1046700096010E9421399B01AC01632D722D812F7F
:10468000902F0E94C935362E272E182F092FA501ED
:10469000940169817D8189859D850E94C9356DC0A0
:1046A0005A962D913D914D915C915D97C701B60150
:1046B0000E9421394B015C0120E030E040E05FE3E3
:1046C0000E94213929813D8149855D850E94CA3535
:1046D000A70196010E9421399B01AC01632D722D27
:1046E000812F902F0E94C935362E272E182F092F83
:1046F000262F372F482F592F6A8D7B8D8C8D9D8DBE
:104700000E94E13818168CF52A8D3B8D4C8D5D8DFD
:104710006AA17BA18CA19DA10E94C9359B01AC011E
:104720000E94CA356B017C0129813D8149855D85E7
:104730006E897F89888D998D0E94CA359B01AC0155
:10474000C701B6010E94C9366B017C01BAA9BD8BB5
:10475000EE89E983FF89FD83288D2987398D3D877F
:104760003A8C2B8C1C8D0D8DC3C0A50194016981E1
:104770007D8189859D850E94CA3569837D8389876E
:104780009D87B6C02E893F89488D598DC701B601D6
:104790000E9421399B01AC01632D722D812F902F36
:1047A0000E94C9355B014C019B01AC016EA17FA148
:1047B00088A599A50E94E13818160CF095C02EA185
:1047C0003FA148A559A5632D722D812F902F0E94DE
:1047D000C9352E893F89488D598D0E94C9366B0194
:1047E0007C013EA02FA018A509A542E04D8B80C0FA
:1047F0005A962D913D914D915C915D97C701B601FF
:104800000E9421394B015C0129813D8149855D85EB
:104810000E94BF3687FF39C020E030E040E05FE310
:10482000C501B4010E9421399B01AC0169817D81E0
:1048300089859D850E94C935A70196010E9421396D
:104840009B01AC01632D722D812F902F0E94C935E1
:104850006FAB78AF89AF9AAF2AA53BA54CA55DA5F4
:104860000E94E13818168CF4A501940169817D81BC
:1048700089859D850E94C93569837D8389879D8748
:104880003FA828AC19AD0AAD33C02AA53BA54CA55D
:104890005DA5632D722D812F902F0E94C9359B013C
:1048A000AC010E94CA356B017C0129813D8149859B
:1048B0005D856BA97CA98DA99EA90E94CA359B0123
:1048C000AC01C701B6010E94C9366B017C01BBA9CE
:1048D000B983ECA9ED83FDA9F9872EA92D873AA408
:1048E0002BA41CA50DA504C03A2C2B2C182D092D8A
:1048F000A7019601C301B2010E94CA352B013C01F8
:104900002E8D3F8D48A159A10E94BF3687FF07C059
:10491000A30192016E8D7F8D88A199A11CC02EA547
:104920003FA548A959A9632D722D812F902F0E9470
:10493000E138181684F52EE333EC4EE259E36E8D20
:104940007F8D88A199A10E94CA356E8F7F8F88A321
:1049500099A3A30192010E94C9356B017C01232D0B
:10496000322D412F502F6AA57BA58CA59DA50E94B5
:10497000BF3687FD11CE89819D81A985BD85809334
:10498000AF039093B003A093B103B093B2033D89FA
:104990003093AA030FC089819D81A985BD8580932D
:1049A000AF039093B003A093B103B093B2034D89CA
:1049B0004093AA03E091ED06F091EE0691899111E2
:1049C00004C080910E0283FF3FC0ABADBCAD5196D9
:1049D0008C915197807349F19E96CD90DD90ED902A
:1049E000FC90D1979923D1F02091C3033091C40357
:1049F0004091C5035091C6036091AF037091B0031D
:104A00008091B1039091B2030E9421399B01AC01C6
:104A1000C701B6010E9421396B017C01C701B601B3
:104A20000E9465028093C7030AC010921702109279
:104A300018021092190210921A021092C703809164
:104A40000E02877F80930E0247E029893A89429FB0
:104A5000F001439FF00D1124ED5EFC4FFA87E987CA
:104A60008091C70386832091A2033091A3034091D4
:104A7000A4035091A503632D722D812F902F0E94C6
:104A8000213969837A838B839C830E94A8366B01CA
:104A90007C0160919E0370919F038091A00390918F
:104AA000A1030E94A8364B015C01A70196010E9458
:104AB000C9350E9442376D837E838F839887ED814D
:104AC000FE81A985BA85ED93FC93EF2B41F480918B
:104AD0000E0281FF04C0816080930E020EC12091FE
:104AE0009A0330919B0340919C0350919D03C30115
:104AF000B2010E94CA352B013C0129813A814B81C8
:104B00005C81C501B4010E94C9359B01AC01C301A0
:104B1000B2010E94C9364B015C0120EC31EE44E643
:104B20005EE40E9421390E94A8360E944237603D0F
:104B300037E073078105910560F4A7E049895A8938
:104B4000A49FF001A59FF00D1124ED5EFC4F15828E
:104B500053C0603ABFE07B078105910560F447E0F0
:104B600029893A89429FF001439FF00D1124ED5E9F
:104B7000FC4F51E011C06034AFE17A078105910527
:104B800068F447E029893A89429FF001439FF00D7C
:104B90001124ED5EFC4F52E055830CC027E0A9893B
:104BA000BA892A9FF0012B9FF00D1124ED5EFC4F76
:104BB00033E03583A7E049895A89A49FF001A59F76
:104BC000F00D1124ED5EFC4F2581022E04C0969558
:104BD0008795779567950A94D2F74D815E8102C0DB
:104BE000440F551F2A95E2F75183408361157105E3
:104BF00051E08507910568F427E0A989BA892A9FC1
:104C0000F0012B9FF00D1124ED5EFC4F7383628346
:104C100004C04FEF5FEF538342838091EC06809393
:104C20003D038F5F863019F08093EC0602C010922E
:104C3000EC06E091EF06F091F006832D922DA12F66
:104C4000B02F868F978FA0A3B1A3C0929E03D0925E
:104C50009F03E092A003F092A10329813A814B8146
:104C60005C81C701B6010E94C935A50194010E946B
:104C7000213960939A0370939B0380939C039093D4
:104C80009D032091AB033091AC034091AD03509153
:104C9000AE03632D722D812F902F0E94BF3681119C
:104CA000A5C820E030E0A901632D722D812F902F3F
:104CB0000E94E13890910E02181614F092FF04C081
:104CC000916090930E0219C01092F0061092EF06B8
:104CD0009091CA038091EB06891709F487C881E097
:104CE000890F803109F480E02091C803921302C03B
:104CF0008093C8038093CA0379C8EC960FB6F894E2
:104D0000DEBF0FBECDBFDF91CF911F910F91FF90FE
:104D1000EF90DF90CF90BF90AF909F908F907F905B
:104D20006F905F904F903F902F900895CF93DF93B7
:104D3000C091EF06D091F0062097C9F080919903B9
:104D40008160809399036091AF037091B00380916B
:104D5000B1039091B2039B01AC010E9421396A8B8F
:104D60007B8B8C8B9D8B1092F0061092EF06DF915F
:104D7000CF9108952F923F924F925F926F927F92C0
:104D80008F929F92AF92BF92CF92DF92EF92FF925B
:104D90000F931F93CF93DF933090EB06311002C037
:104DA000D0E101C0D32DD150C091C803CD1709F473
:104DB00016C1ED2EF12C22E3D29F80011124055360
:104DC0001C4FF801A688B788C08CD18C628D738D7A
:104DD000848D958D9B01AC010E94CA35F801268D0A
:104DE000378D40A151A10E9421394B018C019B01BB
:104DF000AC01B501C6010E94BF3687FD02C0540157
:104E0000680182E38E9DF0018F9DF00D1124E55322
:104E1000FC4FC501D601828B938BA48BB58BD1112E
:104E200001C0D0E1D150CD1307C08091CA03C8138F
:104E300068C00E94962665C022E32E9DC0012F9D6A
:104E4000900D11249C0125533C4F790192E3292EAA
:104E5000AD2EB12C2A9CC0012B9C900D1124FC017D
:104E6000E553FC4F6F01D11101C0D0E1D1508091C9
:104E7000CA038D1302C00E9496262A9C80012B9C97
:104E8000100D112405531C4FF80186889788A08CBB
:104E9000B18CA501940162897389848995890E94E6
:104EA000BF36882359F1F801628D738D848D958DFD
:104EB0009B01AC010E94CA35F801268D378D40A1B7
:104EC00051A10E942139F7012289338944895589EA
:104ED0000E94CA352B013C019B01AC01C501B40104
:104EE0000E94E138F80118162CF4428A538A648A29
:104EF000758A04C0828A938AA48AB58A7601CD1302
:104F0000A7CFF2E3CF9F8001112405531C4FCF5F41
:104F1000C03109F4C0E0D091C80382E3282EC31544
:104F200009F45BC0CC2ED12C2C9CC0012D9C900D83
:104F300011249C0125533C4F7901F8014288538884
:104F400064887588F90182889388A488B588A5014A
:104F50009401C301B2010E94BF3687FF24C0F8014B
:104F6000628D738D848D958D9B01AC010E94CA3535
:104F7000F801268D378D40A151A10E942139A3014E
:104F800092010E94CA352B013C019B01AC01C50175
:104F9000B4010E94E138181634F4F701428A538AAA
:104FA000648A758ADC2F2C9CF0012D9CF00D112455
:104FB000E553FC4F26893789408D518D628973896D
:104FC000848995890E94BF36811101C0DC2FCF5F93
:104FD000C03109F4C0E08701A2CFD093C803DF91AC
:104FE000CF911F910F91FF90EF90DF90CF90BF90E6
:104FF000AF909F908F907F906F905F904F903F9079
:105000002F9008952F923F924F925F926F927F92CE
:105010008F929F92AF92BF92CF92DF92EF92FF92C8
:105020000F931F93CF93DF93CDB7DEB7C454D1094D
:105030000FB6F894DEBF0FBECDBF3B010091EB066B
:10504000202E312C22E3229DA001239D500D1124FE
:10505000BA0165537C4F7AAF69AFFB0111922A9573
:10506000E9F7F3012085FB01218BF3014481558190
:1050700066817781E9ADFAAD46A757A760AB71AB02
:1050800021FF40C02CE0E1EFF1E0DE0159960190F4
:105090000D922A95E1F78BAB9CAB2BE132E03EAB56
:1050A0002DABBE01635F7F4F23967FAF6EAF23971B
:1050B000CE01499621969FAF8EAF2197E2E30E9FD6
:1050C000C00111249C0125533C4F3EAF2DAF685EBB
:1050D0007F4F7CAF6BAF78AF6FAB10E082E3829D08
:1050E0009001839D300D1124C90185539C4FFC0113
:1050F0003C962596FFAFEEAF25972C01F0E14F0EC1
:10510000511C3CC02CE0E1EFF6E0BFCFEDADFEADB1
:105110002193319341935193FEAFEDAF2596EEADC0
:10512000FFAD2597C080D180E280F380C216D30600
:10513000E406F50610F469017A012596EEADFFAD9F
:105140002597C082D182E282F3820E947337A50143
:1051500094010E94C936EFA9F8AD619371938193D0
:105160009193F8AFEFAB20E030E0A9010E94BF3689
:1051700087FD42C01F5F133009F44CC0EBA9FCA9A6
:105180006191719181919191FCABEBABEDA9FEA97D
:1051900081909190A190B190FEABEDABA5019401EF
:1051A0000E9421390E94EE382396EEADFFAD239781
:1051B00061937193819391932396FFAFEEAF239701
:1051C0002196EEADFFAD2197C190D190E190F19085
:1051D0002196FFAFEEAF21976C197D098E099F09CB
:1051E0009B01AC0197FF92CF22273327A901261BF1
:1051F000370B480B590B8ACF112321F0113021F0C6
:1052000080E803C080E201C080E4F2019081892B34
:105210008083B0CFCD28CE28CF2809F496C1CE0107
:1052200085960E94A7314B015C0122E3229DC001BB
:10523000239D900D11249C0125533C4F7901F901C8
:10524000868E978EA0A2B1A2BE016B5D7F4F83E3D5
:1052500092E00E945131F701628F738F848F958F96
:10526000BE016B5D7F4F87E292E00E945131F701F2
:1052700066A377A380A791A7118910FD12C0F3013F
:10528000208131814281538113FD06C0F70122A79D
:1052900033A744A755A709C0C501B4010E9421390D
:1052A000F70162A773A784A795A78091CA0308177F
:1052B00011F011FF0DC082E3829DF001839DF00D7E
:1052C0001124E553FC4F128A138A148A158A54C09C
:1052D0002DEF36E03CAB2BAB8E010F5F1F4FBE01B5
:1052E0006F5C7F4F7AAB69ABC12CD12C76010DABD3
:1052F0001FABEBA9FCA981909190A190B190FCAB60
:10530000EBABEBADFCAD4190519061907190FCAF77
:10531000EBAFA3019201C501B4010E9421399B01A9
:10532000AC01C701B6010E94C9356B017C01A50122
:105330009401C301B2010E94C935F80161937193D0
:10534000819391938F0129A93AA96BAD7CAD261762
:10535000370779F62FEE3FEF4FE75FE3C701B6015E
:105360000E94E13818166CF482E3829DF001839D5F
:10537000F00D1124E553FC4F12A213A214A215A2A2
:1053800071C02FEE3FEF4FE75FEBC701B6010E9400
:10539000BF3687FF11C082E3829DF001839DF00D2F
:1053A0001124E553FC4F89E996E7A6E9BEE782A3FD
:1053B00093A3A4A3B5A356C08DA99FA90E94A7310A
:1053C0006DA97FA983E392E00E9451314B015C01FA
:1053D000A701960160E070E080E89FE30E94C93574
:1053E00020E030E040E05FE30E9421390E94C039B4
:1053F0006B017C0120915002309151024091520288
:1054000050915302C501B4010E942139A7019601B0
:105410000E9421394B015C01A701960160E070E018
:1054200080E89FE30E94C9359B01AC01C501B4012E
:105430000E94C9366B017C0120E030E0A9010E9486
:10544000BF3687FF03C0C12CD12C760182E3829D39
:10545000F001839DF00D1124E553FC4FC2A2D3A2AD
:10546000E4A2F5A282E3829D8001839D100D1124A8
:1054700005531C4FF801818981FD69C089AD9AAD42
:105480000E941C1D6B017C018090090790900A0707
:10549000A0900B07B0900C07A50194010E94E13881
:1054A00018162CF4A5019401C501B40104C0A7018C
:1054B0009601C701B6010E942139F801668B778BEE
:1054C000808F918F82E3829D8001839D100D112436
:1054D00005531C4FF80182A093A0A4A0B5A0A5017C
:1054E000940166897789808D918D0E94E138181624
:1054F0002CF4F801868A978AA08EB18EC092090793
:10550000D0920A07E0920B07F0920C078CE0FE01A4
:10551000B596ADEFB6E001900D928A95E1F78CE07B
:10552000FE013D96A1EFB6E001900D928A95E1F75C
:105530008091C9038093EB068F5F803109F480E08E
:105540008093C9030E94BA2602C080E001C081E0B6
:10555000CC5BDF4F0FB6F894DEBF0FBECDBFDF913F
:10556000CF911F910F91FF90EF90DF90CF90BF9060
:10557000AF909F908F907F906F905F904F903F90F3
:105580002F900895CF93DF930E947F3280E3E8E964
:10559000F3E0DF011D928A95E9F7CFEED2E083E2D6
:1055A000FE0111928A95E9F71092F0061092EF062B
:1055B0001092120310923D0381E08093EC0610924A
:1055C000EE020E944E328091ED028F878BB1837E76
:1055D0009091EC02892B8BB98BB18F719091ED0278
:1055E000892B8BB9DF91CF910895CF93DF93C1E1E0
:1055F000D7E08991882319F00E943D02FACFDF910C
:10560000CF910895CF93DF9321E5829FC0011124AC
:10561000EC01DD5F40E550E0BE0181E197E00E94D2
:10562000731E892B69F4109211070E94020240E553
:1056300050E061E177E0CE010E94B01D80E001C042
:1056400081E0DF91CF9108959FB7F89420911007E2
:10565000822B809310079FBF08959FB7F8942091E5
:105660000F07822B80930F079FBF08959FB7F89471
:1056700080930E079FBF08952FB7F89490910D0760
:105680008095892380930D072FBF08959FB7F894C5
:1056900020910D07822B80930D079FBF0895AF9235
:1056A000BF92CF92DF92EF92FF920F931F93CF930F
:1056B000DF93EC010FE312E05C018CE0A80EB11C5B
:1056C000C990D990E990F99020E030E0A901C70194
:1056D000B6010E94E13818168CF0F8012191319141
:1056E000419151918F01C701B6010E94BF3687FDDC
:1056F00005C0CA15DB0521F780E001C081E0DF911C
:10570000CF911F910F91FF90EF90DF90CF90BF90BE
:10571000AF9008958F929F92AF92BF92CF92DF92F7
:10572000EF92FF920F931F93CF93DF93EB012BE147
:10573000E22E22E0F22E8C016B018CE0C80ED11C0F
:105740006991799189919991F70181909190A190B6
:10575000B1907F010E947337A50194010E94C93660
:10576000F80161937193819391938F01CC15DD05BD
:1057700039F7DF91CF911F910F91FF90EF90DF905C
:10578000CF90BF90AF909F908F9008950E9402029B
:1057900010921602089596B1977082E0982771F0E2
:1057A00081E0292F227091FD80E090FF826021111D
:1057B00001C08460947019F48860089580E00895B1
:1057C0001F920F920FB60F9211242F933F934F9376
:1057D0005F936F937F938F939F93AF93BF93CF9379
:1057E000EF93FF930E94CB2BC82F882389F081FD74
:1057F0000E945F03C3FF05C080910D078260809304
:105800000D07C0FF05C080910D07806280930D07D2
:10581000FF91EF91CF91BF91AF919F918F917F9128
:105820006F915F914F913F912F910F900FBE0F900D
:105830001F9018951092F0019091600297FD03C09F
:1058400090E29093F001882331F09091F00180E292
:1058500089278093F00108958F929F92AF92BF9213
:10586000CF92DF92EF92FF920F931F93CF93DF932C
:10587000CDB7DEB72D970FB6F894DEBF0FBECDBF04
:105880006B017C01042F20E030E0A9010E94BF36AB
:1058900087FF07C08DE20E943D02F7FAF094F7F807
:1058A000F094102F123060F020E030E048EC52E429
:1058B000C701B6010E9421396B017C011250F2CF61
:1058C00000FF0AC020E030E040E251E4C701B60129
:1058D0000E9421396B017C0120E030E040E05FE371
:1058E000C701B6010E94CA350E943B3710E03AE07A
:1058F000832E912CA12CB12C611571058105910588
:1059000091F0EE24E394F12CEC0EFD1EE10EF11C5F
:10591000A50194010E944A3A605DF7016083B901D4
:10592000CA011F5FE9CF80E3101748F4E1E0F0E01F
:10593000EC0FFD1FE10FF11D80831F5FF5CF1013EA
:1059400013C0FE01E10FF11D80E381831F5F0CC0D6
:10595000101303C08EE20E943D02FE01E10FF11D13
:1059600080810E943D0211501111F2CF2D960FB689
:10597000F894DEBF0FBECDBFDF91CF911F910F9185
:10598000FF90EF90DF90CF90BF90AF909F908F905F
:1059900008952091600220FF08C02BE832E441E224
:1059A0005DE30E94213941E001C040E00C942C2CC1
:1059B0002091600220FF08C02BE832E441E25DE361
:1059C0000E94213944E001C043E00C942C2C0F9339
:1059D0001F93CF938C01C0E0F80161917191819187
:1059E00091918F010E94D82CC23019F08CE20E9454
:1059F0003D02CF5FC33081F7CF911F910F91089582
:105A0000CF93DF93843630F06AE00E942A3AC0E3F5
:105A1000C90F03C0C0E08A3030F06AE00E942A3A21
:105A2000D0E3D90F01C0D0E0805D0E943D02DD23AC
:105A300019F08D2F0E943D02CC2329F08C2FDF918D
:105A4000CF910C943D02DF91CF910895CF93DF93D6
:105A5000FC018491EF012196882321F00E943D02F0
:105A6000FE01F7CFDF91CF91089581E693E00C948A
:105A7000262DCF93C82F8AE693E00E94262D8C2FE7
:105A80000E94002DCF910C94352D811104C081E727
:105A900093E00C94262D0C94392DCF93DF93C0E026
:105AA0008C2F0E94022B81110EC0109211078EE3E1
:105AB0000E943D020E94F52A8AE30E943D0287E08F
:105AC0000E94392D12C080911107882371F00E9425
:105AD000E609D82F8EE30E943D020E94F52A8AE350
:105AE0000E943D028D2F0E94452DCF5FC230C1F62E
:105AF000DF91CF910895CF92DF92EF92FF92CF93F3
:105B0000DF93D82F6A017B01C22F84E20E943D02FD
:105B10008D2F0E94002D8DE30E943D024C2FC70166
:105B2000B6010E942C2CDF91CF91FF90EF90DF9077
:105B3000CF900C94352DCF93DF93D82FC62F84E2CE
:105B40000E943D028D2F0E94002D8DE30E943D0298
:105B50008C2F0E94002DDF91CF910C94352DEF9268
:105B6000FF920F931F93CF93DF9360914B0270E0EE
:105B700080E00E949B2D60914E0270E081E00E94C7
:105B80009B2D60914C0270E082E00E949B2D609101
:105B90004D0270E083E00E949B2D6091600262FBE9
:105BA000662760F970E084E00E949B2D609160029E
:105BB00066FB662760F970E085E00E949B2D80916E
:105BC0006002082E000C990B692F661F6627661F5E
:105BD00070E086E00E949B2D60914F0270E08AE0A9
:105BE0000E949B2D409150025091510260915202AF
:105BF0007091530223E08BE00E947B2D4091540270
:105C000050915502609156027091570223E08CE04A
:105C10000E947B2D60916002617070E08DE00E94B7
:105C20009B2D6091600265FB662760F970E084E15E
:105C30000E949B2D6091600263FB662760F970E013
:105C400085E10E949B2D609160026295617070E019
:105C500086E10E949B2D6091610270E087E10E94C5
:105C60009B2D409162025091630260916402709199
:105C7000650223E088E10E947B2D409166025091ED
:105C80006702609168027091690223E089E10E94D5
:105C90007B2D60916A0270916B028AE10E949B2DBC
:105CA00040916C0250916D0260916E0270916F0292
:105CB00023E08BE10E947B2D4091580250915902C4
:105CC00060915A0270915B0220E08EE10E947B2D70
:105CD00040915C0250915D0260915E0270915F02A2
:105CE00020E08FE10E947B2D6091600266956170DB
:105CF00070E080E20E949B2DD4E6F12C0BE112E0D3
:105D000083E0E82EED0ECD2F82E0F81691F0E3E06F
:105D1000FE16E9F0F1E0FF1631F0F8014081518103
:105D2000628173811AC0F80144855585668577853F
:105D300014C020E030E041E655E4F801608D718D3B
:105D4000828D938D0E94C936AB01BC0106C0F8015B
:105D500044A155A166A177A1705823E08C2F0E9421
:105D60007B2D0C5F1F4FCF5FEC12CECFD65FF3942D
:105D7000DC3821F6DF91CF911F910F91FF90EF90CA
:105D800008958DE50E943D020C94352DCF93DF934D
:105D9000CDB7DEB72C970FB6F894DEBF0FBECDBFE0
:105DA00084E693E00E94262D6DEF71E0CE0101960E
:105DB0000E948A2BCE0101960E94E72C8AE30E9462
:105DC0003D0280910F020E94002D0E94C12E2C9650
:105DD0000FB6F894DEBF0FBECDBFDF91CF9108950F
:105DE0001F920F920FB60F9211242F933F934F9350
:105DF0005F936F937F938F939F93AF93BF93EF9333
:105E0000FF9380910A02813049F080910E07811141
:105E100005C00E945F0381E00E94362BFF91EF9145
:105E2000BF91AF919F918F917F916F915F914F91B2
:105E30003F912F910F900FBE0F901F90189593B127
:105E400096718091600286FD02C086E198279923B1
:105E500049F091FB882780F992FD8260907119F0DA
:105E60008460089580E008952F923F924F925F9250
:105E70006F927F928F929F92AF92BF92CF92DF925A
:105E8000EF92FF920F931F93CF93DF93CDB7DEB7BF
:105E9000A1970FB6F894DEBF0FBECDBF90910B0255
:105EA0009111C4C18F8FFE013D9689E0DF011D92E3
:105EB0008A95E9F786E08D8BEBE1F2E0FA8FE98FC6
:105EC0005F019E012A5E3F4F490100E010E0C12CB6
:105ED000D12C76019F8D892F90E09E8F8D8F802F02
:105EE000002321F0013021F090E103C094E001C0D3
:105EF00098E0D4019D934D01ED8DFE8D02C0F59586
:105F0000E7958A95E2F7E0FF1BC020E030E040EC27
:105F10005FEBD50194966D917D918D919C919797B2
:105F20000E942139362E472E582E692EA701960140
:105F30000E94BF3687FD04C0C32CD42CE52CF62C60
:105F40000F5F1F4FB4E0AB0EB11C0330110539F6E3
:105F5000209066023090670240906802509069027B
:105F600084E0A82EBB24B39461EF71E0CE010196CA
:105F70000E948A2B80916102682E712CFE0131965D
:105F800021EF31E03C8F2B8F39A328A3DE015696F9
:105F90004D0180E090E000E010E0B701A6017058EC
:105FA0002D8D3E8D082E02C0359527950A94E2F777
:105FB00020FF22C00F5FA8A1B9A11D921D921D92C2
:105FC0001C9213979301082E02C0359527950A94C9
:105FD000E2F720FF03C0BB2019F007C0BB2029F067
:105FE000C082D182E282F38204C040835183628303
:105FF0007383D4012C91122B0196BFEF8B1A9B0A4D
:10600000349628A139A12C5F3F4F39A328A38330B0
:10601000910531F6602F70E080E090E00E947137CA
:106020000E94C0399B01AC0110931002C201B10162
:106030000E9421396D877E878F87988BBE01635FB1
:106040007F4FCE0101960E94022834E030930E0269
:106050000E94D81E0E94FD34BB20E9F00E941F2F31
:10606000FE01769620E030E090E06191462F4123DA
:1060700059F0AC01022E02C0559547950A94E2F7FB
:1060800040FF02C0609516232F5F3F4F233031053C
:1060900061F7109310020E94D81E80910D0784733F
:1060A00039F110910D0714FF03C086E00E94362BD2
:1060B00015FF03C087E00E94362BB11007C00E9475
:1060C0001F2F9F8D892339F088E003C012FF03C082
:1060D00089E00E94362B80910E07882329F00E94C8
:1060E0005F030E94D81BA2C084E00E943C2B04C026
:1060F000812F8C7109F0B0CF0E94C22A00916A02F0
:1061000010916B020115110549F0AFE9BFE011973D
:10611000F1F700C0000001501109F4CFB1E0BB2637
:10612000C9F020E030E040EA50E460916C027091E8
:106130006D0280916E0290916F020E9421396B0175
:106140007C01209062023090630240906402509083
:10615000650210C0C0906C02D0906D02E0906E029B
:10616000F0906F02209066023090670240906802C3
:1061700050906902AA94A110F7CEE0906102F12C30
:1061800080906C0290906D02A0906E02B0906F02B1
:106190002401350177FA709477F870948D8D9E8D77
:1061A000002E02C0959587950A94E2F780FF2BC0D8
:1061B000C701002E02C0959587950A94E2F7E98DF4
:1061C000FA8D80FF0FC024A135A146A157A1C501BA
:1061D000B4010E94CA35A98DBA8D2D913D914D9182
:1061E0005C9106C02081318142815381C301B2019B
:1061F0000E9421390E94EE38AB8DBC8D6D937D934A
:106200008D939C9313970F5F1F4FEB8DFC8D3496EE
:10621000FC8FEB8F298D3A8D2C5F3F4F3A8F298F62
:106220000330110509F0BACF10920E02A1960FB6F5
:10623000F894DEBF0FBECDBFDF91CF911F910F91BC
:10624000FF90EF90DF90CF90BF90AF909F908F9096
:106250007F906F905F904F903F902F900895EBE666
:10626000F0E08081897E8083E8E6F0E080818E7FA7
:106270008083089584B1897E84B985B1866185B9AA
:106280008091600283FF0BC080916B0086618093D8
:106290006B008091680081608093680008950C9481
:1062A0002F316F927F928F929F92AF92BF92CF9237
:1062B000DF92EF92FF920F931F93CF93DF93EB0147
:1062C0008C015B018CE0A80EB11C89E9682E96E771
:1062D000792E26E9822E3EE7932EC990D990E99037
:1062E000F99020E030E0A901C701B6010E94BF3655
:1062F0008823B9F0A7019601F8016081718182813C
:1063000093810E94C9366B017C01E894F7F89301F0
:10631000A401C701B6010E94E138181614F0360135
:1063200047010C5F1F4FCA15DB05B9F6B301C40165
:10633000DF91CF911F910F91FF90EF90DF90CF9061
:10634000BF90AF909F908F907F906F9008954F92E5
:106350005F926F927F92AF92BF92CF92DF92EF9255
:10636000FF920F931F93CF93DF93EC015C018CE0BE
:10637000A80EB11C8E01C12CD12C7601F8014190E0
:106380005190619071908F0120E030E0A901C3012C
:10639000B2010E94BF36882371F0A3019201C301AC
:1063A000B2010E9421399B01AC01C701B6010E94D4
:1063B000CA356B017C010A151B0501F7C701B6013F
:1063C0000E94C0396B017C019B01AC0160E070E070
:1063D00080E89FE30E94C9362B013C01A301920192
:1063E000688179818A819B810E942139699379939F
:1063F00089939993AC16BD0689F7C701B601DF9161
:10640000CF911F910F91FF90EF90DF90CF90BF90B1
:10641000AF907F906F905F904F9008951F93CF93B0
:10642000DF93142F20E030E040EA51E40E9421394C
:106430000E94A8360E944237EB012097D1F080914C
:106440000B02811116C0111103C00E94D81B06C097
:106450000E94911780910C0281FD0BC02FEF80E705
:1064600092E0215080409040E1F700C00000219769
:10647000E4CFDF91CF911F910895E1EFF1E0A1EF1B
:10648000B6E041915191619171914D935D936D93FE
:106490007D9381E0ED3FF807A1F7089580914C02CC
:1064A000682F20914D02422F982F917080FD94E02B
:1064B000822F817020FD80E261FD986041FD806443
:1064C00062FD906142FD80689093EC028093ED0242
:1064D00008951F920F920FB60F9211248F939F93DE
:1064E0008BB19091EC029C71837E892B8BB915BC8A
:1064F0009F918F910F900FBE0F901F9018958091D4
:106500006F008D7F80936F0080918100887F816014
:10651000809381001092EE0280914E0290910A02C7
:106520008F3F39F420910E07211103C0903881F478
:1065300002C0943069F090E0009741F0EFE9FFE08D
:106540003197F1F700C000000197F6CF81E001C05C
:1065500080E09091600292FF02C091E08927882339
:1065600011F0289A0895289808951F920F920FB657
:106570000F9211242F933F934F935F936F937F93C9
:106580008F939F93AF93BF93EF93FF938091EE020E
:10659000811122C28BB19091FE02907E8F71892B66
:1065A0008BB98BB1837E9091FD02892B8BB9809141
:1065B000FC0286BD82E085BD81E08093EE02789486
:1065C0008091100390911103892B09F0BFC0809135
:1065D000120390913D03981709F4A4C0E0911203AF
:1065E0002E2F30E087E0E89FF0011124ED5EFC4F94
:1065F000F0931103E09310038281938190938900BB
:10660000809388008081918190930C0380930B0389
:10661000E48180910D038E1761F1E0930D0382E117
:10662000E89FF0011124E25CFC4FF0930F03E0932C
:106630000E0384859585A685B785B695A79597950C
:1066400087958093F7029093F802A093F902B09394
:10665000FA028093F3029093F402A093F502B093B0
:10666000F6028093EF029093F002A093F102B093B0
:10667000F202A0910E03B0910F0350969C91509797
:106680008091ED0289278093FE0287E0829FF001CE
:10669000839FF00D1124ED5EFC4F25814D915D919E
:1066A0006D917C911397022E04C07695679557954E
:1066B00047950A94D2F74093FF02509300036093EA
:1066C00001037093020314964D915D916D917C913D
:1066D0001797022E04C076956795579547950A94AB
:1066E000D2F7409303035093040360930503709320
:1066F000060318968D919D910D90BC91A02D04C01C
:10670000B695A795979587952A95D2F78093070315
:1067100090930803A0930903B0930A0386810E9413
:10672000020314C00E947F32E0910E03F0910F0328
:106730008189882339F01092B3008091B0008F775F
:106740008093B00084E00E94462B46C180910902EC
:106750008130B1F486B180729091F001891781F097
:10676000109209028CE0E1EFF1E0ADEFB1E00190B1
:106770000D928A95E1F780910D07806480930D0753
:106780001092FD024091EF025091F0026091F102EF
:106790007091F2028091FF0290910003A091010399
:1067A000B0910203840F951FA61FB71F8093EF02BD
:1067B0009093F002A093F102B093F202E0910E03E5
:1067C000F0910F03448555856685778548175907ED
:1067D0006A077B0768F524E02093FD024485558510
:1067E00066857785841B950BA60BB70B8093EF020C
:1067F0009093F002A093F102B093F202208980916D
:10680000F1019091F201A091F301B091F40125FF03
:1068100004C00197A109B10903C00196A11DB11DD2
:106820008093F1019093F201A093F301B093F401EE
:106830004091F3025091F4026091F5027091F602DA
:106840008091030390910403A0910503B091060386
:10685000840F951FA61FB71F8093F3029093F40235
:10686000A093F502B093F602448555856685778539
:10687000481759076A077B0778F52091FD022860C1
:106880002093FD024485558566857785841B950B8D
:10689000A60BB70B8093F3029093F402A093F5023A
:1068A000B093F60220898091F5019091F601A091B4
:1068B000F701B091F80126FF04C00197A109B109C1
:1068C00003C00196A11DB11D8093F5019093F601BF
:1068D000A093F701B093F8014091F7025091F802AC
:1068E0006091F9027091FA02809107039091080378
:1068F000A0910903B0910A03840F951FA61FB71F2B
:106900008093F7029093F802A093F902B093FA02F1
:106910004485558566857785481759076A077B073B
:1069200078F52091FD0220612093FD024485558574
:1069300066857785841B950BA60BB70B8093F702B2
:106940009093F802A093F902B093FA022089809103
:10695000F9019091FA01A091FB01B091FC0127FF90
:1069600004C00197A109B10903C00196A11DB11D81
:106970008093F9019093FA01A093FB01B093FC017D
:1069800080910A02843039F49091FD0280911002C6
:1069900089238093FD0280910B0390910C03019752
:1069A00090930C0380930B03892B69F410921103CD
:1069B00010921003809112038F5F80931203863030
:1069C00011F4109212039091FD028091EC0289273C
:1069D0008093FD021092EE02FF91EF91BF91AF9173
:1069E0009F918F917F916F915F914F913F912F91E7
:1069F0000F900FBE0F901F9018958091600282FF3C
:106A000002C0289A01C028988091EC028093FD0270
:106A100080914B02880F845081958093FC02809175
:106A20006F00826080936F0008958F929F92AF9263
:106A3000BF92CF92DF92EF92FF920F931F93CF936B
:106A4000DF937C016B01DC01CC91D0E0FE01EF5EB5
:106A5000F84F80818D3229F4EF012296818101E087
:106A600009C08B3219F0CE5ED84F03C0EF012296D9
:106A7000818100E0912CF0E010E020E030E0A901FD
:106A80005E01E0EDE80FEA30D0F4FF5FF93098F4F2
:106A900091101150A5E0B0E00E94723ADC01CB01E8
:106AA000880F991FAA1FBB1F9C01AD012E0F311D1E
:106AB000411D511D0AC0911008C01F5F06C0EE3F66
:106AC00041F4911006C0992493942196D5018C919C
:106AD000D7CFFF2309F44FC0CA01B9010E94713713
:106AE0004B015C0120E030E0A9010E94BF36882301
:106AF00049F11F3F64F42AE037ED43E25CE3C5014E
:106B0000B4010E9421394B015C011E5FF2CF1F3F8F
:106B100059F42DEC3CEC4CEC5DE3C501B4010E9452
:106B200021394B015C010EC0112361F020E030E0FF
:106B300040E251E4C501B4010E9421394B015C01DE
:106B40001150F2CF002351F0B7FAB094B7F8B094D7
:106B5000F60180829182A282B38206C0D6018D9214
:106B60009D92AD92BC921397C151D740C150F7018D
:106B7000C08381E001C080E0DF91CF911F910F9130
:106B8000FF90EF90DF90CF90BF90AF909F908F904D
:106B900008955058BB27AA270E94E1350C947B38F2
:106BA0000E94423838F00E94493820F039F49F3F63
:106BB00019F426F40C9418380EF4E095E7FB0C94C5
:106BC000E937E92F0E94A03858F3BA176207730714
:106BD0008407950720F079F4A6F50C94DA380EF4C2
:106BE000E0950B2EBA2FA02D0B01B90190010C01DD
:106BF000CA01A0011124FF27591B99F0593F50F4F5
:106C0000503E68F11A16F040A22F232F342F44274C
:106C1000585FF3CF469537952795A795F040539544
:106C2000C9F77EF41F16BA0B620B730B840BBAF014
:106C30009150A1F0FF0FBB1F661F771F881FC2F77F
:106C40000EC0BA0F621F731F841F48F48795779593
:106C50006795B795F7959E3F08F0B0CF9395880F4D
:106C600008F09927EE0F9795879508950E9442386E
:106C700060F080E891E009F49EEF0E94493828F026
:106C800040E851E071F45EEF0CC00C9418380C949D
:106C9000DA38E92FE0780E94A03840F3092E052A5F
:106CA000B1F3261737074807590738F00E2E07F8B3
:106CB000E02569F0E025E0640AC0EF6307F800947E
:106CC00007FADB01B9019D01DC01CA01AD01EF93B7
:106CD0000E94E0360E947B380E9479365F915523EE
:106CE00039F02BED3FE049E450FD49EC0C94CA35F6
:106CF0000895DF93DD27B92FBF7740E85FE31616CD
:106D0000170648075B0718F4D92F0E94E6389F93AF
:106D10008F937F936F930E94003AEEE0F1E00E9420
:106D20001B380E947B382F913F914F915F910E94B9
:106D30003439DD2351F09058A2EA2AED3FE049ECC6
:106D40005FE3D0785D270E94E135DF910C947B38BA
:106D50000E94C23890F09F3748F4911116F40C94B9
:106D6000DB3860E070E080E89FE3089526F01B16B2
:106D7000611D711D811D0C94EF370C940A380E941F
:106D8000C53708F481E008950E945238E3950C94C9
:106D90008C380E94DD360C947B380E94493858F0BC
:106DA0000E94423840F029F45F3F29F00C94E93703
:106DB00051110C94DB380C9418380E94A03868F3F9
:106DC0009923B1F3552391F3951B550BBB27AA27A4
:106DD00062177307840738F09F5F5F4F220F331FDE
:106DE000441FAA1FA9F335D00E2E3AF0E0E832D0A6
:106DF00091505040E695001CCAF72BD0FE2F29D0A9
:106E0000660F771F881FBB1F261737074807AB077A
:106E1000B0E809F0BB0B802DBF01FF2793585F4FEF
:106E20003AF09E3F510578F00C94E9370C94DB382A
:106E30005F3FE4F3983ED4F3869577956795B795D1
:106E4000F7959F5FC9F7880F911D9695879597F9DC
:106E50000895E1E0660F771F881FBB1F6217730755
:106E60008407BA0720F0621B730B840BBA0BEE1F6A
:106E700088F7E09508950E9442376894B1110C9408
:106E8000DB3808950E94A83888F09F5798F0B92FF2
:106E90009927B751B0F0E1F0660F771F881F991F4F
:106EA0001AF0BA95C9F714C0B13091F00E94DA38DF
:106EB000B1E008950C94DA38672F782F8827B85FEF
:106EC00039F0B93FCCF3869577956795B395D9F7A7
:106ED0003EF490958095709561957F4F8F4F9F4FB1
:106EE0000895E89409C097FB3EF4909580957095BD
:106EF00061957F4F8F4F9F4F9923A9F0F92F96E906
:106F0000BB279395F695879577956795B795F1117A
:106F1000F8CFFAF4BB0F11F460FF1BC06F5F7F4F17
:106F20008F4F9F4F16C0882311F096E911C0772329
:106F300021F09EE8872F762F05C0662371F096E832
:106F4000862F70E060E02AF09A95660F771F881F01
:106F5000DAF7880F9695879597F908950E94C238B9
:106F600090F09F3748F4911116F00C94DB3860E0F4
:106F700070E080E89FEB089526F41B16611D711DDB
:106F8000811D0C94EF370C940A38990F0008550FA7
:106F9000AA0BE0E8FEEF16161706E807F907C0F09F
:106FA00012161306E407F50798F0621B730B840BA7
:106FB000950B39F40A2661F0232B242B252B21F481
:106FC00008950A2609F4A140A6958FEF811D811D21
:106FD000089597F99F6780E870E060E0089588233E
:106FE00071F4772321F09850872B762F07C0662302
:106FF00011F499270DC09051862B70E060E02AF0C3
:107000009A95660F771F881FDAF7880F96958795F0
:1070100097F908959F3F31F0915020F48795779527
:107020006795B795880F911D9695879597F908955F
:107030009FEF80EC0895DF93CF931F930F93FF9200
:10704000EF92DF927B018C01689406C0DA2EEF018B
:107050000E943439FE01E894A5912591359145911E
:107060005591A6F3EF010E94E135FE019701A801B9
:10707000DA9469F7DF90EF90FF900F911F91CF9115
:10708000DF91089500240A941616170618060906BB
:10709000089500240A94121613061406050608958E
:1070A0000C9418380E94A838D8F3E894E0E0BB2785
:1070B0009F57F0F02AED3FE049EC06C0EE0FBB0F02
:1070C000661F771F881F28F0B23A6207730784078C
:1070D00028F0B25A620B730B840BE3959A9572F702
:1070E000803830F49A95BB0F661F771F881FD2F740
:1070F00090480C940C38092E0394000C11F488234A
:1071000052F0BB0F40F4BF2B11F460FF04C06F5F5F
:107110007F4F8F4F9F4F0895EF93E0FF07C0A2EA84
:107120002AED3FE049EC5FEB0E94E1350E947B389D
:107130000F90039401FC9058EBE3F1E00C94163AA5
:1071400057FD9058440F551F59F05F3F71F0479518
:10715000880F97FB991F61F09F3F79F087950895FD
:10716000121613061406551FF2CF4695F1DF08C01C
:10717000161617061806991FF1CF86957105610539
:10718000089408950E94A838A0F0BEE7B91788F4C3
:10719000BB279F3860F41616B11D672F782F8827FC
:1071A000985FF7CF869577956795B11D939596393A
:1071B000C8F30895E894BB2766277727CB0197F992
:1071C00008950E94C53708F48FEF08959B01AC0124
:1071D00060E070E080E89FE30C94C9360E94A83814
:1071E00058F19E5760F19851A0F0E9F0983020F5E1
:1071F000092E9927660F771F881F991F0A94D1F7C8
:1072000012C0062E672F782F8827985F11F4000C84
:1072100007C0993FB4F38695779567959395D9F70D
:10722000611D711D811D3EF490958095709561954D
:107230007F4F8F4F9F4F089568940C94DB380C94C8
:10724000DA380E9434390C947B380E94423838F086
:107250000E94493820F0952311F00C94E9370C94E2
:10726000183811240C94DB380E94A03870F3959FD5
:10727000C1F3950F50E0551F629FF001729FBB272D
:10728000F00DB11D639FAA27F00DB11DAA1F649FC9
:107290006627B00DA11D661F829F2227B00DA11D7C
:1072A000621F739FB00DA11D621F839FA00D611D02
:1072B000221F749F3327A00D611D231F849F600D23
:1072C000211D822F762F6A2F11249F5750409AF04C
:1072D000F1F088234AF0EE0FFF1FBB1F661F771FD8
:1072E000881F91505040A9F79E3F510580F00C94A3
:1072F000E9370C94DB385F3FE4F3983ED4F386958E
:1073000077956795B795F795E7959F5FC1F7FE2B42
:10731000880F911D9695879597F908950E94A83832
:10732000E8F09E37E8F09639B8F49E3848F4672FB5
:10733000782F8827985FF9CF8695779567959395ED
:107340009539D0F3B62FB1706B0F711D811D20F4EC
:1073500087957795679593950C94EF370C940A3839
:107360000C94DB389F930E9452380F9007FCEE5F1D
:107370000C948C3819F416F40C9418380C940A38C0
:107380000E94A838B8F39923C9F3B6F39F57550B59
:1073900087FF0E940F3A0024A0E640EA900180583F
:1073A0005695979528F4805C660F771F881F20F00C
:1073B00026173707480730F4621B730B840B20290C
:1073C00031294A2BA69517940794202531254A2761
:1073D00058F7660F771F881F20F0261737074807D2
:1073E00030F4620B730B840B200D311D411DA095F1
:1073F00081F7B901842F9158880F96958795089544
:107400009B01AC010C9421390E94C23830F09F37A7
:1074100010F40C94DB380C94EF370C940A3891502C
:107420005040660F771F881FD2F708959F938F9360
:107430007F936F93FF93EF939B01AC010E942139DF
:10744000EF91FF910E941B382F913F914F915F91D7
:107450000C942139991B79E004C0991F961708F004
:10746000961B881F7A95C9F780950895AA1BBB1BA8
:1074700051E107C0AA1FBB1FA617B70710F0A61B34
:10748000B70B881F991F5A95A9F780959095BC0155
:10749000CD010895A1E21A2EAA1BBB1BFD010DC050
:1074A000AA1FBB1FEE1FFF1FA217B307E407F507B4
:1074B00020F0A21BB30BE40BF50B661F771F881F90
:1074C000991F1A9469F760957095809590959B0126
:1074D000AC01BD01CF010895EE0FFF1F0590F4919F
:1074E000E02D09940E947D3AA59F900DB49F900DC8
:1074F000A49F800D911D11240895A29FB001B39FF8
:10750000C001A39F700D811D1124911DB29F700DAC
:10751000811D1124911D0895FB01DC0104C08D9192
:107520000190801921F441505040C8F7881B990BF5
:067530000895F894FFCF5E
:00000001FF
